:020000041100E9
:10300000002370B5284C0120636101F031FA4020A3
:103010000223FE21254A207401F0B0FA002833D1A2
:103020000223FF21224A207C01F0A8FA00282BD19C
:10303000204BA2899A4224D1E3891F4A93420CD1A2
:103040001E4B63611E4B2268002A03D1002B01D066
:1030500023CB23C401F080FA70BD1A4A934201D0F9
:103060000023F0E7184B194A1B68934205D9C02288
:103070000421207C920001F0FBFA104B6361144B99
:10308000E1E700232374EBE7CC223820AC21920146
:10309000207401F0EDFA0028F3D10E4B63610E4B62
:1030A000E3810E4BCFE7C0468463FF1F9063FF1F91
:1030B0009263FF1F5959000083050000D14200119F
:1030C00050BA001182150000A863FF1F871300008B
:1030D0005CBA00116D430011AAAAFFFF44BA0011A7
:1030E000F7B5164B0192C318021D002000938823E8
:1030F0005B05D3181B685C1C1AD09CB2402C18D8F6
:103100008D781E0CAC466746CD782D023D43AE420D
:1031100006D1019800280ED110000C70240A4C70C2
:1031200003249BB20733A343D218009B9A42DED3F9
:10313000FEBD4432F9E71000FAE7C046FC0F00007C
:10314000802213B503000324019189B25201073193
:103150009B18A14304305A1A88235B05C3181B68C7
:10316000591C03D190429241104016BD99B240299A
:1031700007D80B000733A343C0189042ECD30020BC
:10318000F3E74430F9E7134B134A1B68126810B594
:10319000FA24934201D81A00F824104BE4021B6869
:1031A0009A4210D813000E4A12689A420ED3013385
:1031B00007D1F823DB029C4203D10A49054808F0F5
:1031C000EBFA200010BDFC24E402ECE7FE24E4024C
:1031D000F7E7C04600C0071100D0071100E0071153
:1031E00000F00711FFFFFF7FF0B59BB015000490C2
:1031F0000391402A00D9A0E006AB59801A80FFF75E
:10320000C2FF0400042816D9002206A9FFF768FFB0
:10321000052810D906AB1B88AB420CD1002D07D076
:10322000514B2A000499C01808F086FB002802D1EF
:1032300001201BB0F0BD06AB1D8020000699FFF7F2
:103240007FFF041E7BD1069B0793FFF79CFF802323
:103250005B01C618802307001B039E4201D3F8269A
:10326000F60288235B05F31801931B68013302D033
:10327000019808F021F83D49019808F08DFA3B1DAE
:103280000293331D05938822029B52059B181B68ED
:1032900008935A1C3CD044219AB20091402A04D889
:1032A0000320D11D814389B2009103991B0C8B42ED
:1032B00024D0402A22D80122300008A9FFF710FFAD
:1032C000021E1BD1380008A9FFF70AFF04000428DA
:1032D00031D9009A059B9B1880225201B218934263
:1032E00040D288235B05C118009A09A808F054F859
:1032F0001D4B009A09A9F01808F09EF9009A029B4C
:103300009446634402931A4B029AFB189A42BAD32A
:1033100088235B05FC1821680198013908F03CFA04
:10332000200007F0C9FF039A07AB5A8030000799C5
:10333000FFF706FF0400002C03D1002079E70428E2
:10334000FBD988235B05E018069908F025FA0323CA
:10335000EA1C9A4300D16BE7034B0499E01808F08C
:103360006BF965E70424ECE704000011FFFFFF7F21
:10337000F80F0000F7B505001400402A21D80027F7
:1033800001AE71803780FFF7FEFE042816D93A009F
:103390003100FFF7A5FE042810D93688BC420BD0B7
:1033A000BD4209D0221CB44200D9321C064B92B255
:1033B000C118280007F0F0FF30B2FEBDC04300B2D4
:1033C000FBE703204042F8E70400001137B5042270
:1033D00004000D0001A81649FFF7CCFF02000428E5
:1033E0000BD1019BA34208D3AB4204D0104901A8E2
:1033F0000195FFF7F9FE01203EBD0E4C2368200029
:10340000019307F059FF019920000139019108F05B
:10341000C3F980235B01E418074B9C42EED10422E0
:10342000034901A80195FFF7DFFE0020E4E7C0464D
:103430005555000000C007110000081130B589B0D3
:1034400008F06AF910226946254808F02DF8254B46
:10345000009A9A420ED1019B029A0F2B33D8002179
:1034600001240698013B08D2002900D00292029B59
:10347000013331D10023029325E0551CF2D1020023
:103480002100EFE710341022200004A908F00CF806
:10349000029B013301D1069B0293882304995B05AB
:1034A000C918059B06981A03120B049105928142D4
:1034B00003D02B4201D107F06FFF019B013B019329
:1034C000019B002BDED1029B002B03D004930498B8
:1034D0004168084709B030BDE025014C2D03EFE7F6
:1034E0000000011150485936F7B50F490F4B0A68D3
:1034F00004001A4084235B0013430B60030003277E
:103500001033019300252E00112008F01DFA084BFE
:103510001B683B40AB4002351E43202DF4D1019B7C
:1035200040C4A342EED1F7BD5CF0004000FEFEFFB8
:1035300064F00040802270B5AD4CAE4BD20000214B
:1035400020001C6008F0C8F92300AB4A88331A60D9
:10355000AA4B1A786E23002A00D01133E3620A23A3
:103560002365A74B1878A74BA0630138E361C3B26A
:10357000032B01D810232362A34B37226361C82396
:10358000DB00A36123008C331A60082336210F3A35
:10359000E518E16323646264E9670439251DE9677E
:1035A00025003B26BC352E602500C0352B6025004C
:1035B000C4352A6025000636CC352E602500083E2D
:1035C000C8352E602500D03529602100D4310B602C
:1035D0002100D8310A6021000225E0310D6025006C
:1035E0004221DC35296025001B3EE4352E60250094
:1035F000E8352B602500EC352A6022000525F432E1
:1036000015602200F03211602200183190321160F2
:1036100022009432136023003C2298331A60AF23B7
:10362000DB002360794B2363032805D808F024F9D5
:10363000330235371523636096232100FA225B009D
:10364000A360E360C8332361714BFC319200A36433
:103650000A6062626F4A704DA2627322E2656D3A3F
:103660006265A2650232E5644A60022161669621C4
:103670008900A166626709210022E166A2676749A5
:10368000674A684E2167E2673560032811D808F061
:10369000F3F896089EA61023CDE70E23CBE70C2364
:1036A000C9E720001A259C30056020000735A030AE
:1036B00005602000A83003602300FA20F833800062
:1036C000186023006420A433186023005F38AC33F3
:1036D000186023000338B03318602300C630B433B9
:1036E000186023000020B833186023003825FC330D
:1036F0009D604D4D5A665D644C4D9A64DD61962522
:10370000AD001D624A4D9A675D62F53DFF3D9D62C9
:103710001E25484ADD6618675867D9651966DA6755
:10372000BE23C021444A5B00E250444B4900635031
:1037300004316250C4225200A350FA23E4205B00FB
:103740000432A3500432A3503D493E4A3E4BD1605F
:103750003E49800019503E49E938FF3819503D492B
:10376000043019503C491038D1613C4911633C493F
:1037700051633C4911603C49195019003B48F831EC
:1037800008603B49D16582213A4A89005A501A00A3
:1037900039490832D1671A003849B432116088219A
:1037A000374A89005A501A00364988321160364A21
:1037B000DA6408F0A1F8012007F0DEFD70BD2000FA
:1037C00014259C30056020000435A03070E72000EF
:1037D00010259C30056020000335A03068E72000EC
:1037E0000E259C30056020000235A03060E7C04601
:1037F0000004FF1F5866FF1F5071FF1F1846FF1F70
:103800004A0AFF1F3A07000080C3C9019A0200005C
:1038100050C300006A180000280A0000204E000073
:1038200088130000F009FF1F00400011681000001D
:10383000C4090000DC05000040420F001027000012
:10384000FD1BFF1FFC00FF1F0000FF1F252FFF1F98
:103850004D32FF1FE530FF1FD91FFF1FF51FFF1F50
:10386000A121FF1F491FFF1FC528FF1F8D2CFF1F10
:10387000D918FF1FD127FF1F3925FF1F4525FF1F1F
:10388000491EFF1F011FFF1FC11DFF1FF7B50B0CB6
:10389000FF270122009300233C001E001D009446D8
:1038A000019089B262469A401000084018413618CB
:1038B000B6B2FF2F02D1012E00D19FB20098024074
:1038C0001A41AD18ADB2FF2C02D1012D00D19CB22E
:1038D0000133102BE6D10320012E07D1012D04D195
:1038E000019B2401E4191C700138FEBD102EFCD18F
:1038F0000238102DF9D00230F7E710B5064C2378C6
:10390000002B07D10548FFF7EFFD0548FFF7ECFD59
:103910000123237010BDC0461866FF1F2C66FF1FD1
:103920001C66FF1FF0B58BB00D000123019010291C
:1039300036D8FFF7E2FF00231A001B48C15C0133B1
:103940005218102BFAD1023B002A29D0174B184CE1
:103950001F68002306A9E25C1600FA5C56405E541C
:103960000133102BF7D102AA07F00EFE2A0002A99C
:10397000019807F091FD07F037FF23681B182360BB
:1039800007F032FF63681B18636007F02DFFA36820
:103990001B18A36007F028FFE3681B18E3600023EF
:1039A00018000BB0F0BDC0462C66FF1FB844FF1FC7
:1039B0001C66FF1F0223F0B501245F4D5F4E2B7084
:1039C0005F4B91B01C705F4F0393336808207B708E
:1039D00006F036FA0023984205D07A78552A02D0AC
:1039E000332A00D09CE03360002006F0C1FC07F0D1
:1039F000CBFEFFF79FFD07F067FD1F22012400218A
:103A0000514B10AE1A70514B1C70514B1970514BE9
:103A100019689143163A0A431A6060221968914363
:103A2000403A0A431A6007F06FFE07F0CDFCC12050
:103A3000FF21494B80001A588A431A50C522920030
:103A400098588843BF3901439950985843490840D2
:103A50008021C9010143802099509958C00509026D
:103A6000090A0143995080213D48490107F09CFC17
:103A7000032322003B49019400933B4807F07CFE5E
:103A80002C223A4905A807F087FC05AC617820781C
:103A9000023406F0FBF9A642F8D10121002006F01D
:103AA0000FFB0121092006F00BFB314B314A19684D
:103AB00003201140A022D2020A431A608022196812
:103AC00092040A431A6019682B4A1140802292031B
:103AD0000A431A60294B2A4A934200D8012007F072
:103AE0009BFE07F041FD07F09FFD287807F014FCCE
:103AF000039B1878C0B207F0DFFE07F0F5FC214900
:103B0000042007F0F1FD06F0FFFB00F0AFF800F035
:103B1000DDFD00F06BFE00F019FA002011B0F0BDE1
:103B200000932100174A042007F0FEFB8023DB05E9
:103B30009C62FFF783FC57E74A0AFF1F34F00040FE
:103B40001846FF1FB463FF1F480AFF1F490AFF1FE3
:103B5000680AFF1FBCF0004000E100E0FF00FFFF2B
:103B60001C46FF1FA058FF1F1C56FF1F68B90011FD
:103B700014F00040FF7FF8FFFFFF9FFF5071FF1F11
:103B80000080FF1F3B00010870B500252849294A25
:103B900029484D6308CA1B051B0DED188242F9D157
:103BA0000022264B8B63264B08211A628022254B6C
:103BB0009205DA67244BDA688A43DA60234A12787E
:103BC000012A03D09A6822490A409A600121EE2412
:103BD0002048E40002686C438A430260DA681120DE
:103BE0008A43DA6007F0A0FE112007F0EDFC1120F7
:103BF00007F06AFE184A200C0400642390420AD899
:103C0000FA220023D200904205D9144B0A21C01891
:103C100007F0EAFBC3B2124A1372124BD4801B782E
:103C2000002B04D1104B1021187807F0D5FC70BD83
:103C3000000005408805054000060540FF01000022
:103C400000F0004004E100E03CF000404A0AFF1FA1
:103C5000FFDFFFFF00380040B70B000030F8FFFF28
:103C60009C63FF1FD865FF1FD463FF1F002210B5A0
:103C70001100112007F0D8FD10BD0000F8B5002399
:103C800001250826394F3A4C3B62E3681120AB43CB
:103C9000E360E368B343E36007F096FC112007F0AC
:103CA00043FE112007F068FC4023226829001343DB
:103CB000236080236268DB02134380226360A36871
:103CC00007201343A360A3682A4A1340A3608023FC
:103CD000A2689B0113431022A360236C93432364C7
:103CE000236C2B43236480235B003B62226B224BBB
:103CF0001A402263626B1A406263A26B1A40A2638D
:103D0000E26B1340E3631D4AE3681340E36006F08F
:103D1000A7F92900072006F0D3F98021184A1120BD
:103D2000536C0B43536407F04FFDFD21154B164AAE
:103D300089005A508023C720626B5B03134363637F
:103D4000E36880003343E360E368104A1D43104B8F
:103D5000E56019581140802212020A431A5080224D
:103D600092051A600B4B5E63F8BDC04600F0004040
:103D70003CF00040FFFFDFFFEFFFEFFFFFFF7FFFA3
:103D8000003800400000FF1F893B0011FF00FFFFCB
:103D900000E100E00000054030B503A804880B20D6
:103DA000002C0ED14968074D087849780902014373
:103DB0000A20A94205D1012120001980024B1B7A5B
:103DC000137030BD192A00009C63FF1FF7B5150062
:103DD00008AA16884A680F4F1478527812022243B4
:103DE0000A24BA4214D10122DBB2019200962A00C1
:103DF00007F0DAF9041E0BD1074B1B68002B07D024
:103E000068782A78000210434242504101309847B6
:103E10002000FEBD022900002063FF1F30B50125F0
:103E200003790400BFB02B4212D00A49408806F043
:103E300027FD28420CD06A46074B69465B8D5580AA
:103E40001380064B60881B7A1371002203F0DEFD9D
:103E50003FB030BD1863FF1F6042FF1F9C63FF1F10
:103E600010B50549054806F0C1FC0421044A05487F
:103E700006F07EFC10BDC0461863FF1FFFFF000068
:103E800094B900116042FF1F10B5024804F040FCD5
:103E900010BDC0461D3E0011062310B583701033BF
:103EA0000371443B43712A3383714433C37100234C
:103EB0000222012103720E4B027041701C88817234
:103EC0004472197A0273C1729A784273DA788273F3
:103ED0000322C2731A7902745A7942740C228274D2
:103EE0009A79C274DB7903751123C370152010BD54
:103EF0009C63FF1F10B5142007F016FB124B142211
:103F00000021186007F0E8FC002007F04DFB0120BD
:103F100007F0CAFB022007F0A7FA032003F09CFE7B
:103F2000042005F0B1FE052003F0DAF8062003F0C6
:103F3000A7FD072001F03CF9082006F0F9FB092055
:103F400000F028FF10BDC0462463FF1F10B507F026
:103F50004BFB012007F0C8F907F016FA002010BD4E
:103F6000094B10B50400984205D0012904D1200066
:103F7000064906F03BFC10BD0229FCD1013904F0D2
:103F800085FB0028F3D0F6E7FEFF00004A63FF1F21
:103F900030B5012503790400BFB02B4218D00D497C
:103FA000408806F06DFC284212D06A460A4B0B4945
:103FB0001B8813800A235380293313716B4609220F
:103FC000581D07F0E9F900226946608803F01EFDDC
:103FD0003FB030BD4A63FF1FFE42FF1F9C63FF1FBF
:103FE00070B50D7A100004AA2C0016881022144017
:103FF000154220D1002E20D10A78022A18D14A6811
:10400000517815780E4A09022943914205D00D4A8C
:10401000914209D01C800A2404E014220A491A8023
:1040200007F0BAF9200070BD0C2208491A80F7E7A2
:104030001C800124F6E70824F4E70B24F2E7C046CD
:10404000F3FF0000F4FF00009C44FF1F74BA00114E
:1040500010B504000749084806F0C8FB074804F0FB
:1040600097FA0020E40704D50721054A054806F021
:104070007FFB10BD4A63FF1FFFFF0000613F00117F
:10408000D8B90011A442FF1F00B50C4BBFB01A787D
:104090000B4901A800F0DCFB6B4680B25880002879
:1040A00009D06A46074B69461B881380064B0022DD
:1040B000188803F0ABFC3FB000BDC0462863FF1F6B
:1040C0002963FF1FFE42FF1FFE43FF1F00B50C4B7D
:1040D000BFB01A780B4901A801F0DEFB6B4680B235
:1040E0005880002809D06A46074B69465B8D1380CB
:1040F000064B0022188803F089FC3FB000BDC04683
:104100005263FF1F5363FF1FA442FF1FFE43FF1FA5
:10411000F7B50E00377A1C0008AB11003D001A8875
:1041200020231D401F423CD13378022B3BD17368C2
:104130001F785B781B023B431E4FBB4208D01E4FCB
:10414000BB4214D01D4DAB4221D00A252800FEBD34
:10415000002A2AD1142C2AD82200F06807F01CF972
:10416000174B1C70012CF1D9FFF7B0FFEEE7002AC6
:104170001BD1202C1BD82200F06807F00DF9114B41
:1041800004211C70104B187807F026FADEE7E3B222
:104190000124009201940A00310007F005F805009F
:1041A000D4E70825D2E70125D0E70B25CEE70D257A
:1041B000CCE7C046F3FF0000F4FF00000229000036
:1041C0005263FF1F2863FF1FD463FF1F10B502480F
:1041D00004F09EFA10BDC046913F001170B5160064
:1041E00004AA148805AA15784A6850781178000244
:1041F0002A4A0843801805284BD807F03DFB0313D3
:104200001E29343F0720042C0BD80522121BAA427A
:1042100000D92A0022491A803000091907F0BCF899
:10422000002070BD0720112CFBD81222121BAA42BD
:1042300000D92A001B491A80EEE707200E2CF0D87F
:104240000F22121BAA4200D92A0017491A80E3E75D
:104250000720032CE5D80422121BAA4200D92A0009
:1042600012491A80D8E70720032CDAD80422121B3F
:10427000AA4200D92A000E491A80CDE70720032C54
:10428000CFD80422121BAA4200D92A0009491A8059
:10429000C2E700220A201A80C3E7C046DCD5FFFF30
:1042A00023BA00117063FF1F13BA00110EBA001178
:1042B00009BA001104BA001110B50D21024A0348D1
:1042C00006F056FA10BDC046F8B900111443FF1F9E
:1042D00037B5002000F0CCF8204D214BEA89287C2E
:1042E0009A422AD1042201A900F076F9040000F0D4
:1042F00033F9002C30D16B4699882B68C9BA4B43EF
:104300002989184A1B145B1853806B46D9886B683F
:1043100049BA89B24B4369891B0C5B181248191CB6
:104320001BB2834200DD011C0B0400D50021138861
:1043300091800133138020003EBD0223002101AA99
:1043400000F01CF96A46040002230121287C063291
:1043500000F014F90443CAE70124ECE78463FF1F6B
:10436000830500009C63FF1F0F27000037B5012065
:1043700000F07EF81F4D07226946287C00F02CF9DA
:10438000041E33D16B461B787F2B2FD800F0E4F846
:104390006B46D878F02302041B031A406B469B88B7
:1043A00015495BBA9BB21A432B68000953432A890B
:1043B0001B0C9B184B806B465A789B7812031B0191
:1043C0001A436B68024353436A891B0C9B180B48C2
:1043D0001A1C1BB2834200DD021C130400D500220C
:1043E0000B888A8001330B8020003EBD00F0B4F8BA
:1043F0000124F9E78463FF1F9C63FF1F0F27000060
:1044000010B50F4C237C002B0CD0382B0BD1012086
:1044100000F02EF8CC22AC21207C920100F028F98B
:1044200000F09AF810BD074BE2899A42FAD10120B8
:1044300000F01EF80021207C00F0FAF8F0E7C046FA
:104440008463FF1F8305000010B5084B1A7C002A07
:1044500009D05B69002B06D09847041E01D0FEF7F7
:10446000CFFD200010BD0124F9E7C0468463FF1F83
:1044700070B500210600162005F05EFE0121152012
:1044800005F05AFE07F018F80400092007F074F848
:1044900000222B4B2B4DDA6661321A6019685B3AA9
:1044A0009143002E28D0023A0A431A60AC4209D147
:1044B0000A22DA6107321A6200221A639A63013211
:1044C000DA6370BD204A944203D11E22DA610532BC
:1044D000F1E71E4A944203D13022DA610632EAE75C
:1044E0001B4A944203D14322DA610832E3E7194AB6
:1044F0009442E1D16922F7E702220A431A60462278
:10450000AC4203D0104A944204D194225A6106323C
:104510009A61D1E70D4A944201D1E622F6E70C4AAE
:10452000944204D13422FF325A610D32F0E7094A35
:104530009442C1D1E62252005A610A32E8E7C046ED
:10454000005000400024F4000048E801006CDC0248
:104550000090D00300D8B80510B50024064B092000
:10456000DC6607F031F82100162005F079FD210006
:10457000152005F075FD10BD00500040F8B51C0079
:104580000023134D0F00EB666860160007F0C4F8B7
:1045900001238022EB6623002F615200013B08D2E9
:1045A00006F04AFF08200B4A1168002C03D12000B6
:1045B000F8BD2A61F2E72B6F034203D02B69013C5F
:1045C0003370013613685B1A032BEED90124EEE732
:1045D000005000406008FF1F002370B5124D14000A
:1045E000EB6668600E0007F097F801238022EB6607
:1045F00023005200013B08D206F01EFF08200B4AA0
:104600001168002C03D1200070BD2A61F2E72B6FE6
:10461000034203D02B69013C3370013613685B1AE7
:10462000032BEED90124EEE7005000406008FF1F85
:10463000002370B50C4C0D00E366606007F06CF869
:104640000123E366256106F0F7FE8020074A80001B
:104650001168636B034205D113685B1A032BF8D909
:10466000012070BD0020FCE7005000406008FF1FE3
:10467000002370B5134C0E00E3666060150007F070
:104680004BF80123E36626610F33626B1A42FCD0BC
:104690002B0A23611023626B1A42FCD0EDB2256114
:1046A00006F0CAFE8020084A80001168636B03424E
:1046B00005D113685B1A032BF8D9012070BD0020C7
:1046C000FCE7C046005000406008FF1F10B5084CD2
:1046D000E368002B08D1074B1B685B045B0C0A33B3
:1046E0006360054B1B68236006F02EFEA06010BDC2
:1046F000C463FF1FC8F00040CCF0004010B507F0C5
:104700000BF80F4B996A9A6A8A42FBD10D4C62688A
:10471000A0688A18121A531E884200D31300A160A1
:104720002168DA0B52185B0407495B0C6360226056
:104730000B60064B1A6006F07FFE206810BDC04675
:1047400000F00040C463FF1FC8F00040CCF0004000
:1047500070B51D4C23793F2B01D93F2323711B4B8F
:1047600022791A701878C0B206F056FE182318493C
:10477000184A0B80184913800B805380A37917497E
:1047800080200B800C21938001334B430001191CC6
:10479000834200D9011C124BD18019806379002B10
:1047A00001D101336371237A012B01D802232372D3
:1047B0006279237A0B4853430A21584306F014FECA
:1047C000094D286070BDC046B863FF1F480AFF1F2F
:1047D000FC43FF1FC445FF1FFA43FF1FA465FF1FD3
:1047E000F843FF1F71020000A863FF1FF8B51021F6
:1047F0000020FEF7EBFD114C011E114D09D10C22DA
:10480000104BC1CBC1C4280007F066F8FFF7A0FF2A
:10481000F8BD0C2220000C49FEF7ACFD0C2802D09C
:10482000084B43CB43C40C2228000849FEF7A2FDE5
:104830000C28EBD00C220021E5E7C046B863FF1F2F
:104840008463FF1F68BA0011FC0C0000F50C000027
:10485000F0B5002504000E0085B0AA4263D04B1CC1
:10486000087801934B788978377909021943F378EE
:104870003F061B040B431F430397207065702528D8
:1048800000D173E012D810280AD806F0F5FF46E7E9
:104890002C2C2C87958E2C2C2C2C2C2C2C2CC700C3
:1048A000232800D1A9E0FF23637094E0562857D055
:1048B00010D8332800D199E0552837D02628F2D1D6
:1048C000914B2900132218001D0007F005F8FEF790
:1048D00097FB5AE0722800D17FE0DC2800D1D6E0B7
:1048E000712800D16FE0DB2800D0EBE0042ADAD990
:1048F0001025052A05D0551F2A003800711D06F025
:104900004BFD05223100200006F046FD2A0039004B
:10491000601D06F041FD053505E00C2220007B49B5
:1049200006F03AFD0C25280005B0F0BD013A784D9F
:104930000C2A13D8002A0AD02800019906F02CFD71
:10494000FFF706FF0C2228007249FEF74DFC2900F4
:104950000C22601C06F020FD0D25E4E70C22EBE79D
:104960006B4D6D4B2A0043CB43C2E9E7013A664DDC
:104970000C2A11D8002A08D00199280006F00CFD55
:104980000C2228006549FEF72FFC29001322601C29
:1049900006F002FD1425C6E70C22EDE7052260496A
:1049A000601C06F0F9FC0625BDE712225D49601C7B
:1049B00006F0F2FC1325B6E708225B49601C06F0FE
:1049C000EBFC0925AFE77178F72900D96BE7574B66
:1049D000188801F0BDFB0225A5E7554B012A03D03D
:1049E00072781A706270F6E71B785DE70922514908
:1049F000601C06F0D1FC0A2595E7042A04D94E4D27
:104A00002F6006F0A1FCA860FFF778FE0422039057
:104A100003A9601C06F0C0FC052584E7474D062A63
:104A200015D906222800019906F086FF00280ED02D
:104A300006220199280006F0AFFC06224049280012
:104A4000FEF7D2FB01233A4A11780B431370290079
:104A50000622601C06F0A0FC072564E7931E394E71
:104A60001A2B0CD8551E2A000199300006F094FC30
:104A70003549AAB23000FEF7B7FB00F049F9334BD5
:104A800031001D78601C6A1E06F086FC4BE7022A86
:104A900000D808E77378BFB26370B378A370032AB5
:104AA00005D0033A390092B2F01CFEF79DFB1022AC
:104AB0003900E01CFEF75EFCC51C002800DB32E775
:104AC000607088E7DA2800D0EDE6042A00D8EAE62C
:104AD000082A15D9B37972791B021343F2791204AB
:104AE0001A43337A1B0613433B603B6805223100AF
:104AF0002000039306F050FC0422601D03A95EE72A
:104B0000FE236370F1E7C0468463FF1F74BA00118F
:104B1000B863FF1FFC0C000068BA0011F50C000020
:104B20009063FF1F7063FF1F3845FF1FFE43FF1F89
:104B3000B463FF1F9C63FF1FC463FF1F6509FF1F52
:104B4000ADAC0000B765FF1FAEDE0000B565FF1F0E
:104B500070470000020010B5094B0A32094C92B2AE
:104B6000DA815A8298811882207802F057F904225B
:104B7000054B012120781A7006F02EFD10BDC046AD
:104B8000C244FF1F0266FF1F0166FF1F013870B598
:104B9000042809D806F070FE0309200812001C4BF7
:104BA0000221187806F018FD70BD194B08211878FD
:104BB00006F0C2FC0022174B1A72F5E70024154BD1
:104BC000134D082128781A681C8106F055FC210035
:104BD000287806F019FEE7E70D4B0821187806F053
:104BE000ABFC0D48FFF758F90C4B0D4A9B799380AD
:104BF0000C4A13808022074B52001A810A4B1B7803
:104C0000002BD1D0094A136006F0FEFCCCE7C04669
:104C1000D463FF1FA863FF1F0744FF1FB863FF1F74
:104C2000C445FF1FA465FF1FB463FF1F34F000409D
:104C300010B5002903D10920013105F041FA10BD5A
:104C400010B501290DD10021092005F039FA054BD5
:104C50001B78002B05D02622034B04485A72FFF71D
:104C600079FF10BDD865FF1FA863FF1FC4090000AE
:104C70000300F0B50A4D8E18B14202D152008018DF
:104C8000F0BD0C782F6824093C5D0F271C700C7850
:104C900001313C402F683C5D5C700233ECE7C0465C
:104CA000F443FF1F0E22114B10B51A700D23104C48
:104CB00010492370093A043B0F48637006F06CFBFF
:104CC0002D2301220D490E48E371FFF7D1FF012288
:104CD0000C49FFF7CDFF01220B49FFF7C9FF002266
:104CE0000A491000FEF780FA10BDC046D465FF1FC8
:104CF000B565FF1F23BA0011B765FF1F6709FF1FC6
:104D0000BD65FF1F6609FF1F6509FF1FAEDE0000BE
:104D100010B51D2207480849FEF72CFB002805DDC9
:104D20000922064B013018705A7010BDFFF7BAFF08
:104D3000FBE7C046B765FF1FAEDE0000B565FF1F8D
:104D400010B5114B1A781870002A0ED000280BD11C
:104D50000E4B1A78062A07D85423D340DB0703D515
:104D60000B4B187802F05AF810BD0028FCD0074B06
:104D70001B78012B02D0033B022BF5D8044B0121F9
:104D8000187806F029FCEFE7D865FF1F0166FF1FC2
:104D90000266FF1FF8B5534E534A5449307008203D
:104DA00005F090FA0121092005F08AF9092005F0A3
:104DB00073FA0121002005F083F9002005F06CFA58
:104DC000FEF71EF906F0F8FC032249494948FFF7AF
:104DD0004FFF2D24030004221C7047490130FFF7C8
:104DE00047FF30230470454D454C437083702E3B84
:104DF000062220004349EB87FEF7BCFA062813D0B1
:104E0000200006F099FC022809D00321200006F0BA
:104E100023FD8D23E3706E3B2371193363710622EA
:104E200020003849FEF7E0F9374B1B68FC335C641F
:104E3000FFF76EFF0020FFF783FF344F344A012154
:104E4000344B1278387801F0ABFF334C334B0021F0
:104E50001A783878230001F0A3FF01222178304B23
:104E600001391A7000202F4AC9B205F09FFB2E4B62
:104E70005B78552B31D13C222C4B5A722C4A2D4B4E
:104E8000AA81EB812A826B822021307806F03CFDDA
:104E90000120404205F0D6FB0120404205F072FCA3
:104EA000FFF70AFAFEF7DCFF00F08EFC012040421B
:104EB000FFF7CEF8012006F0E7FBF72001F02CF910
:104EC0000121307806F088FB307802F003F91A48A7
:104ED00006F022FBFEF7D2FEF8BDFA22174B520174
:104EE000CEE7C046D463FF1F314C0011414C001186
:104EF0003845FF1F7063FF1F9063FF1FC244FF1FF1
:104F00006509FF1FADAC00005866FF1F0266FF1F5A
:104F10002644FF1F0744FF1FB565FF1FD465FF1F11
:104F2000A665FF1FB765FF1FB463FF1FA863FF1FC0
:104F3000C4090000CE090000D663FF1F4A1F00000D
:104F4000F8B50A0020230D001A40194241D04C4BFD
:104F50001B78002B2CD0FFF7D1FB4A4B4A4C4B4E11
:104F600099686268737A8A1ADB039A4202D3616095
:104F7000FEF784FE327A217A531EDBB299421AD1AF
:104F8000FFF73EFA637A002B0FD0013BDBB263726E
:104F9000002B0AD13E4B5B78552B01D106F034FB38
:104FA000642370795843FFF7D5FD237A01332372C8
:104FB00020206840F8BD9142E4D300232372FFF71C
:104FC00043FA344F3800FEF767FF390006F0C4F9A2
:104FD000D8E70BB2002B0ADA2F4B187806F00CFA40
:104FE000002801D006F0A0FB80200002E1E70224A7
:104FF000214206D0244B01201A72FFF7A1FE2000A7
:10500000D7E70B071BD5FFF779FB1E4B1E491F4C3B
:1050100098684A68637A821ADB039A4202D348602E
:10502000FEF72CFEFFF710FAFFF7EAF900F0E6FBB7
:105030002368DB0701D5FFF7C9F80820B9E710247A
:105040000E002640214206D00D4B1B78002BD6D1F6
:10505000FEF71AFFD3E70124214209D00F4800F0E0
:105060006BF806F0A9FA3100092005F029F8C6E727
:1050700004240800204021429CD0FFF705F8BEE739
:10508000D865FF1FC463FF1FA863FF1FB863FF1F1E
:10509000B463FF1F0744FF1FD463FF1FEC43FF1FD0
:1050A000F0B51B4B1B4F1B883A8804001A4E1B4D52
:1050B00085B09A420DD832889A420AD3184B1A8882
:1050C0002B889A4205D1174A174B12881B889A429F
:1050D0001BD0052001F076F83B8802AA13803388A4
:1050E000019053802B88114D93800F4B02A91B8890
:1050F000D3800F4B2A78188802F092FD0D4B0821BF
:105100002878019A1C7006F0FFF805B0F0BDC04683
:10511000A265FF1FFC43FF1FFA43FF1FA465FF1F8B
:10512000A065FF1F9E65FF1FF843FF1F0266FF1F5C
:10513000FE43FF1F9C65FF1F13B50C4B1C78002C12
:1051400011D1002801D00A4B18600A4A0A4B117885
:105150000A4A10780A4A01920A4A0092002205F08F
:105160001DF9200016BD1124FBE7C0460166FF1F94
:105170009865FF1F0066FF1FF065FF1F0266FF1F97
:10518000DC65FF1FE065FF1F10B5064B12201B7882
:10519000052B06D1044B13221988044B187801F013
:1051A000EDF910BD0166FF1FFE43FF1F0266FF1FE2
:1051B00010B500240122114B52421870104B1C7084
:1051C000104B1A8001F086FF04220F4B21001A7049
:1051D0000E480C3206F080F9102221000C4806F02F
:1051E0007BF907220B4B1C600B4B1C700B4B1C708C
:1051F0000B4B1A700B4B1C7010BDC0460266FF1F94
:105200000166FF1FFE43FF1F0066FF1FF065FF1FC3
:10521000E065FF1FDC65FF1FB465FF1FB365FF1F5F
:105220000044FF1FB265FF1FF8B5174C0600257834
:1052300006A814240078052D23D1B41F134FA5B25E
:105240001824BD421DD88D1FADB2BD4219D8FA2514
:105250006D00AA4215D21D000D4F0A3DADB2BD42F0
:105260000FD80C4C26800C4C21800C4900240A805D
:105270000B4A1380FFF714FF0A4B0421187806F03D
:105280005BF92000F8BDC0460166FF1F790C0000E5
:10529000750C0000FC43FF1FFA43FF1FA465FF1FAE
:1052A000F843FF1F0266FF1FF0B50BB20D0089B077
:1052B000002B00DB70E1A44E307806F09DF8041E50
:1052C00050D00378A22B00D122E1D02B1AD0912B01
:1052D00045D143780E2B42D19C4B82889A423ED1D5
:1052E0009B4A83681278052A39D1032018567F28F3
:1052F00035D0984B1B68002B31D05B68002B2ED02B
:1053000098472CE08078072829D806F0B5FA0428B9
:10531000183F3F74A8D86378002B0CD101218C4B27
:1053200019708D4B1A78002A5BD08C4B307801F0C5
:1053300037FD002855D00722854B1A7051E061785F
:105340000029F8D1E378002B11D0854A854B1278DB
:10535000307801F025FD60706378002BEBD12000E0
:1053600006F0E2F980200002684009B0F0BD784BF9
:105370001B78022BF3D00121307806F00DF90028BC
:10538000EAD10121307806F027F9E5E76378002BB0
:10539000D1D16F4F032807D13B78052B02D10133C0
:1053A0003B701EE00223FBE76F4B1A886F4B0293A2
:1053B000002A0BD01B78002B03D00121307805F098
:1053C000A3FF3B78062B04D1013BE9E7029B1A704F
:1053D000F7E7042B41D10121029B3078197006F0C8
:1053E000FBF85C4B1B68002BB9D01B68002BB6D0B8
:1053F000574A107884E76378554F002B27D106224F
:10540000211D5B4805F0C8FF62895A4B5A491A8032
:10541000A2895A4B1A80E3890B80052139705849BB
:105420000A80584A1380228A574B1A80574B1B78A0
:10543000012B09D11F2000F0C5FEFA229200424341
:105440000421307805F060FF0022484B75E7312BCE
:1054500000D070E70022454B1A700323A0E7062214
:105460000021434806F038F80023454A0421138000
:10547000444A30781380444A138006F05DF80821CE
:10548000307806F059F8A379083B5A425341304A24
:1054900003331370304B1B78002B06D0334B30781E
:1054A0001A78002A06D001F0B9FC0122314B524291
:1054B0001A8096E70121197006F08EF8F5E70821A9
:1054C000307806F039F86378002B00D047E72C4B92
:1054D0002D4F0293E388029A04211380294B3078E0
:1054E00003932389039A138063893B8006F054F861
:1054F000002800D033E7264B1B68002B00D12EE795
:10550000039902983A88098800881B68984726E71B
:105510004379132B00D022E70389012B0AD11D4BBD
:105520001B78022B06D10821307806F005F8FFF72A
:105530002BFE14E7052000F045FE0821020030781C
:1055400005F0E2FE0BE7C0460266FF1F05140000EF
:105550000166FF1F9865FF1F2644FF1F0744FF1FBA
:10556000D465FF1FB565FF1FD665FF1FD865FF1FF8
:10557000A765FF1FFE43FF1FAE65FF1FB065FF1F3E
:10558000A265FF1FA065FF1F9E65FF1FA665FF1F89
:105590009465FF1F9C65FF1F8020C001014200D061
:1055A000E2E6CB0731D5324B1B78002B1DD0314EB4
:1055B00005AC3378052B1AD1023B23702E4B21000A
:1055C0001B7823722D4B1B7863722D4B187801F0DA
:1055D0008BFB002809D007202A4B30701B68002B5A
:1055E00003D01B68002B00D098470120BCE60E209A
:1055F000254B06221B7825492370254B1B786370A9
:1056000002ABC01805F0C8FED8E702230800184016
:10561000194209D0174B1B78052B03D11D4B188855
:1056200006F04AF802209FE60424214203D0FFF747
:1056300037FD200098E6082308001840194200D1E1
:1056400093E6154B1C78012C03D0022C0DD00820BA
:105650008AE6124B124A134913481B88128809889C
:1056600000880094FFF7E0FDF1E7FFF78DFDEEE71E
:10567000D865FF1F0166FF1F0044FF1FB265FF1FB3
:105680000266FF1F9865FF1FB465FF1F0144FF1FDF
:10569000B365FF1FFE43FF1F9C65FF1FF843FF1FFD
:1056A000A465FF1FFA43FF1FFC43FF1F10B502A8AC
:1056B00004880B20002C10D1496808784978090229
:1056C00001430C48814209D1022119800A4B5988B3
:1056D0001170DB7800205BB2537010BD074C0A20BC
:1056E000A142FAD102211980034B998811705B798C
:1056F000F0E7C0466E2A00009C63FF1F6F2A00007F
:10570000F7B5150008AA16884A680F4F1478527822
:10571000120222430A24BA4214D10122DBB20192BE
:1057200000962A0005F040FD041E0BD1074B1B68B4
:10573000002B07D068782A7800021043424250417B
:10574000013098472000FEBD022900001466FF1FAB
:1057500030B5012503790400BFB02B4227D015498D
:10576000408805F08DF828420DD06A46124B6946F4
:105770005B8D138002235380104B5B88938060887D
:10578000002202F043F90E49608805F079F8C0075D
:105790000DD56A460B4B69461B8813800223538044
:1057A000064B9B8893806088002202F02FF93FB05F
:1057B00030BDC0460C66FF1F2844FF1F9C63FF1FBF
:1057C0000466FF1F8244FF1F10B5074C07492000E5
:1057D00005F00CF82000064905F008F80721054AF5
:1057E000054804F0C5FF10BDFFFF00000C66FF1F59
:1057F0000466FF1FF4BA00112844FF1F10B50248C9
:1058000002F086FF10BDC046515700110200F0B5EE
:1058100001270A480A4E51188B1A002B00DCF0BDF4
:10582000082415784308684038404000805B013CFC
:1058300058406D08002CF5D10132EDE7FFFF000064
:105840000EBB0011F0B500250F269D4200DBF0BD18
:105850004C5D070944403440A400A058013578400D
:10586000F3E70000F0B589B06A460D000B000F2782
:10587000110010351C780133260024093E401670B3
:1058800054700232AB42F5D12023024AFFF7DAFF0F
:1058900009B0F0BD14BB0011F0B54E780B7889B09B
:1058A00036020C00170001901E43012A61D9954B66
:1058B0009E4200D877E001339E421CD1062A17D1C0
:1058C000CA788B7812021A430B791B0413434A7966
:1058D00012061A438C4B5A6100221A705A808B4A66
:1058E0005A608B4A9A608B4ADA60002009B0F0BD9A
:1058F00088225205EEE7884B9E423CD182498B7844
:10590000002B00D0F6E00C2A31D10F22A37893436C
:10591000E2781202134322791204134362791206C9
:1059200013434B60E279A07912020243207A00040B
:105930001043627A12060243CA60E27AA07A120227
:10594000024376484A81834208D804236E491422D0
:1059500001980B7005F020FD1420C7E71201D21842
:1059600089235B059A42F0D801238B70BDE7022A98
:10597000FAD00523EAE76A4A01239642E6D1FFF707
:1059800003FC052F0CD9E378A2781B02134322797C
:1059900012041A4363791B061343624A039313608C
:1059A00005F032FEA1E7584D2B78002B9DD1AB7846
:1059B000002B00D1A0E02B8901339BB20093B342AE
:1059C00000D091E0132AD4D9CF7C8B7C3F021221E6
:1059D00020001F43FFF71AFF874200D08EE0002E01
:1059E0003DD1E378A2781B0213432279E9681204BF
:1059F0001A4363791B06134303930A228B4212D185
:105A0000FF23A370E370237163716B89002B09D1AD
:105A1000E37B227C1B0212041343A27B13431B096A
:105A200001336B8100226B89002B8ED0002A67D155
:105A3000686837013818000B6B69000303909842BF
:105A400005D9686105F038FCEB780133EB706868C4
:105A50001022A11C381805F0EFFD2E8145E76F8953
:105A6000009A7B1E9BB293423AD1E278A37812024D
:105A70001A43237905A81B04134362796C68120644
:105A80001A43EB6800920392211D0C22049305F047
:105A900083FC0120260004A940421036FFF7E2FEF5
:105AA000013F012F17D1009A0B232861824200D0B9
:105AB0004CE704221C49200005F0BEFD042203A986
:105AC000686805F0D1FDE968039AFF23914200D18F
:105AD0003CE7F73B3AE73100FFF7C4FE1036DFE75B
:105AE0000923B742A4D831E7009BB34200D9FCE6B2
:105AF00007232BE7022329E7032327E7062325E7CC
:105B00000A2323E7FFFE00009C44FF1F0000011151
:105B1000FFFF00005048593601FF0000FFFF001151
:105B200002FF000034F00040A844FF1F10B5034CF2
:105B30000B000122210000F06BFA10BDED5C00119A
:105B40000B8870B506000D000224162B11D92B000E
:105B50000322094900F05CFA041E0AD1074B2A8887
:105B60001B88191C934200D9111C300089B200F027
:105B7000EFFA200070BDC046195D00117266FF1F6C
:105B800010B54A780400013A0B000220012A07D818
:105B90000A78002A04D005222000024900F038FAD1
:105BA00010BDC046475D00110A7810B50B00040017
:105BB0000220002A04D007222000024900F028FA1F
:105BC00010BDC046F35D00110A7810B50B0004004B
:105BD0000220002A04D009222000024900F018FA0D
:105BE00010BDC046595E001110B5034C0B000B22CE
:105BF000210000F00DFA10BD895E001110B5034CB4
:105C00000B000D22210000F003FA10BDFB5E001115
:105C100010B5034C0B000F22210000F0F9F910BD64
:105C2000555F00110A7810B50B0004000220002A0D
:105C300004D011222000024900F0EAF910BDC0464C
:105C4000655F0011002310B51322190000F0E0F980
:105C500010BD000010B5034C0B001722210000F00E
:105C6000D7F910BDB75F0011002310B51922190034
:105C700000F0CEF910BD000010B5034C0B001B2244
:105C8000210000F0C5F910BDF15F0011F7B584895E
:105C90000D0006000121002C22D000238268D3567B
:105CA0001778002B1EDA0C2C1AD90C3CA4B213194D
:105CB00040880093230002F086FE431E9841013085
:105CC0007B06DB0F6B703F23013C1F40A4B22870A2
:105CD000AF70AC80002C07D0B3680133AB600021FB
:105CE0000800FEBD0020EBE7AC60F8E70B7803701E
:105CF0004B8843704B881B0A83700B79C370042058
:105D000070470420022B06D10020537811781B0223
:105D1000009A0B43138070470B8803700B881B0A93
:105D20004370022070470420009983420AD15378BF
:105D300010781B0203430B80D37890781B02034337
:105D400000204B807047F8B50D004B7801240021EE
:105D5000461C03702B788B4201D82000F8BD6B786D
:105D6000B01C4F1C012B10D1890069184B880222EE
:105D700033704B88B9001B0A7370691805F08CFBEF
:105D800004360434A4B2F9B2E4E7122359436B1881
:105D90005A88043132705B8810221B0A73706918AC
:105DA00005F07AFB12361234ECE770B5049D14004E
:105DB0001E00052B01D8042070BD637812781B02E9
:105DC00013432B80E378A2781B02134302226B80DB
:105DD0002A71211D681D063E05F05EFBB2B22A81C4
:105DE000F02AE8D82800A11D0A3005F055FB002054
:105DF000E2E7002310B50A789A4201D8900010BD5E
:105E00009A008A185488013304705488DBB2240A3B
:105E10004470948884709288120AC2700430EAE751
:105E200010B51100029C062B04D004201022142B64
:105E300001D010BD022222714B7808781B02034367
:105E40002380CB7888781B02034363800431601D74
:105E500005F022FB0020ECE710B50C788B780431BC
:105E60005C43E4B203702200013005F015FB601CB6
:105E700010BD0420022B06D10020537811781B029C
:105E8000009A0B431380704710B50C000A8802314A
:105E900005F002FB208810BD70B504000D000498C9
:105EA0001100012B01D8042070BD1678527812021F
:105EB000324302800200F83255701470E825002C3D
:105EC00000D10C35023B9AB24280AA42EBD8023193
:105ED000043005F0E1FA0020E6E70420009983424F
:105EE0000AD1537810781B0203430B80D378907843
:105EF0001B02034300204B80704710B50C000A883A
:105F0000023105F0C9FA208810BD000070B50121EA
:105F10001E000420049C0E400B4218D1CB40DDB281
:105F20008D4214D90A49DBB2098899420FD3230064
:105F3000F6331D703300580011184978165C0902B9
:105F4000314301332152D9B28D42F4D8002070BDC3
:105F5000BC44FF1F10B50C000A88023105F09CFA02
:105F6000208810BD10B50C788B7804315C43E4B206
:105F700003702200013005F08FFA601C10BD10B5CF
:105F800011000298032B01D8042010BD1478527818
:105F9000043B120222430280CA788C781202224308
:105FA00042809AB28280F22AEED80431063005F09F
:105FB00073FA0020E9E710B50C000B8803700B881A
:105FC0001B0A43704B8883704B881B0AC3708A88F6
:105FD0000430063105F060FAA088043080B210BDAC
:105FE0000420012B03D100201378009A137070470E
:105FF00010B50C000B8803700B881B0A43704A888D
:106000000230043105F048FA6088023080B210BDD9
:10601000F0B589B003931E4B029242000700D05A9C
:10602000019102F020F81325061E2DD0029B0124B9
:106030000370019B002B04D00019039998470019A5
:1060400084B26B461B7A5BB2002B0FDA102138004A
:1060500002F01CFB1925002813D130003219E1B2DF
:1060600002F066FC051E0CD10C34A4B2042304AA71
:10607000380005A993800696948101F0AFFD051EB6
:1060800002D0300005F028F9280009B0F0BDC04664
:106090007066FF1F70B505000C0000280CD00020B2
:1060A000814209D010222000044905F0F5F90120B1
:1060B0002B7823736B78637370BDC04654BB00119B
:1060C000F0B506000D0017001C0085B002291BD09A
:1060D0000020102907D1022B07D0102B03D115E087
:1060E0000020102C08D005B0F0BD69463800FFF73D
:1060F000D1FF2A0069460BE069463000FFF7CAFF6E
:1061000022006946380004E0022BE9D12A00390058
:10611000300005F099FAE6E7031CF72800D9F723C9
:10612000032008499AB2013A0B80D317034006496D
:106130009B189B100B80D30F04499B185B100B809E
:106140007047C046C044FF1FBE44FF1FBC44FF1F32
:10615000034B1B888B4202D3024B4000C152704755
:10616000C044FF1F7066FF1F014B4000185A704764
:106170007066FF1F1722014B1A8070477066FF1F61
:1061800070B505000E2005F0A7FA041E13D0D02329
:10619000037000230622837007494570033005F021
:1061A0007BF9064B2100DA8A62811B7E2373044B44
:1061B000187805F051FA70BD8C66FF1F7C66FF1FD2
:1061C0001045FF1F262803D8024B4000C05A7047D5
:1061D0000148FCE7C244FF1FFFFF000070B5060046
:1061E0000C00094D1C220021280005F075F9074B11
:1061F0001E70074B1C7005F07FF90123002801D0A9
:10620000002312202B7070BD7C66FF1F1045FF1FFE
:106210009D66FF1F70B505000D4C0800E260A1608F
:1062200010220021656005F05FFB012803D11021D9
:10623000A06802F058FD10220021280005F054FB50
:10624000012803D11021606802F04DFD70BDC046E9
:106250007C66FF1F70B5041E05D1002903D00622FD
:106260000D4805F019F90D4B1D78012D11D1002CA9
:1062700005D102221A7005F03FF8280070BD0022F7
:106280001A70074B1B78FF2BF7D02000FFF778FF21
:10629000F3E70025F1E7C0468C66FF1F7C66FF1F11
:1062A0001045FF1F030010B5002801D1002010BDCC
:1062B00000780B4A002803D15988D1821B791376C4
:1062C0001378022BF2D10023984200D103331370CC
:1062D000044B1B78FF2B01D0FFF752FF0120E6E7AC
:1062E0007C66FF1F1045FF1F002911D000280CD02D
:1062F0004B79012803D140225242134303E03F224D
:106300001340032802D001204B7170474022F4E76C
:106310000800FAE770B5094D0100287800280BD075
:10632000074C0622200005F0B7F821002878FFF777
:10633000DBFF200005F018FA70BDC0469C66FF1F09
:106340007666FF1F00290AD0012808D13F224B7929
:106350009343C02B03D0403B5A425341981C704793
:1063600070B5174D06002B78FF2B15D00A2005F0CD
:10637000B3F9041E10D0D0230370C83B8370114BB7
:1063800011491B784670C3700622043005F084F86A
:106390002100287805F060F90C4B1B78012B0DD1FA
:1063A0000B4B1B68002B03D09B68002B00D0984739
:1063B000084B04211878084A05F05EF870BDC04605
:1063C0001045FF1F9C66FF1F7666FF1F9866FF1F24
:1063D000C466FF1FC866FF1F60EA0000014B986893
:1063E0007047C0467C66FF1F014BDB68186870472A
:1063F0007C66FF1F074B10B5DA6813680133136022
:10640000054B1878FF2803D08021C90105F0E4F876
:1064100010BDC0467C66FF1F1045FF1FF7B50E007C
:1064200002F0C8F8051E1CD00E4B06621F78002F24
:1064300000D10778AB791020019305F04DF9041EC7
:106440000FD0D0230380C73B8370019BE91DC3702D
:106450000622043005F020F821003800E66005F03F
:10646000FBF8F7BD0E45FF1F014B18787047C0467B
:106470009C66FF1F054B002805D1054B1A78054B7C
:10648000002A00D1014B18007047C0468C66FF1FE0
:106490009C66FF1F7666FF1F014B58687047C04619
:1064A0007C66FF1F024B1868431E9841C0B27047BC
:1064B000A066FF1F421E03000120152A03D9FF3BDF
:1064C0005A425341D8B27047F0B51C0000230E0069
:1064D00085B0039002920B70029A934201D3002080
:1064E00019E0E55C5A1CD2B2002DF8D0029851197F
:1064F0008142F4DC0233DFB2A35C18000193FFF7A2
:10650000D9FF002807D0013D019A0399EBB23370FF
:106510008A4202D1E01905B0F0BDDB19DBB2DBE73E
:1065200010B50C0002F09EF803001220002B03D0DF
:106530002100588804F090FF10BD000070B50E4D8A
:1065400084006359002B15D0186A002801D004F08C
:106550009BFF2B59586A002801D004F095FF2B5956
:10656000986A002801D004F08FFF285904F08CFFAE
:1065700000232B5170BDC046AC66FF1F1C4B70B58D
:1065800004000E00150099420AD11A4B1B68002B1B
:1065900001D1122070BD1B68002BFAD09847F9E793
:1065A000154B994215D1134B1B68002B0AD01B6861
:1065B000002B07D09847002804D1104B1C70104BBB
:1065C0001D70E7E729002000FFF7AAFF0028E1D1AE
:1065D000F3E7080001F0EEFF0028DAD0037803208B
:1065E000A342D7D12900300004F036FFD2E7C046DD
:1065F000FEFF0000A866FF1FFFFF0000A566FF1F4B
:10660000A466FF1FF7B50400808801F0D3FF0025C2
:10661000A84203D00578A08802F008F81C4E337811
:10662000002B1FD0AB421DD11A4B28001978FFF761
:1066300077FF002818D000233370A3790820A778AB
:10664000A688019305F048F8011E0DD0D0230370F1
:10665000CA3B8370019B477086808371280004F0D9
:10666000FBFF01E0002DE8D1A0880B4B8200D3583E
:10667000002B01D0FFF762FF1721A088FFF768FD0C
:10668000A08801F027FDA08801F0FEFDF7BDC046FF
:10669000A566FF1FA466FF1FAC66FF1FF0B587B09D
:1066A0001D000CAB1B88070001930DAB1B88142049
:1066B00002930EAB1B88160003930FAB1B8800914F
:1066C000049310AB1B88059305F006F8041E1AD03E
:1066D000D0230370CB3B47708370C670062229001D
:1066E0000430002D11D004F0D7FE019B21006381FE
:1066F000029B0098A381039BE381049B2382059B5B
:10670000A37404F0A9FF07B0F0BD04F0E5FEECE7C8
:10671000F7B5009308AB1B8807000C200D0016008E
:10672000019304F0D9FF041E13D0280001F042FFAA
:1067300000280FD00078D0232370C93BA370009BA2
:1067400021002381019B6770A580E680638104F0AE
:1067500083FFF7BD014B1878EDE7C0461045FF1FDA
:1067600013B5040064890389C2888188C0780094C5
:10677000FFF7CEFF13BD000010B5044C20680028C1
:1067800003D004F081FE0023236010BDB066FF1F1C
:10679000A122F0B5818892004A43384B384F1B68DC
:1067A00004009B189D2292009B18827989B01A6080
:1067B0003B68002B5FD01D78324B1B68002B04D048
:1067C0005B68002B01D00020984726000836310076
:1067D000E079FFF7B7FD237DE0710200E0780493D4
:1067E000638A29000393238A0293E3890193A38890
:1067F00000933300FFF752FFE378002B0BD1E289BF
:10680000A379A18802920196E279280000920122E0
:1068100001F0DAFEE0703B68002B20D0FFF7ACFF00
:10682000194D287800281AD0184B1978FFF778FEF0
:10683000002814D02B78E67808200793A78804F066
:106840004BFF011E09D0D0230370CA3B46708370F2
:1068500087808671079804F0FFFE00232B701721B4
:10686000A088FFF775FCA08801F034FCA08801F037
:106870000BFD09B0F0BD064B9DE7C0463409FF1F74
:10688000B066FF1FC466FF1FA566FF1FA466FF1F3B
:106890001045FF1FF8B5070008000E0001F08AFE42
:1068A000041E18D02620FFF78DFC051E00D1257888
:1068B000062004F011FF041E0DD00021062204F072
:1068C0000BFED0232370C23B21006770A370A6800B
:1068D000E8B204F0C1FEF8BDF0B585B001930AAB93
:1068E0001B78070002930BAB1B7808000D00009289
:1068F000039301F05FFE061E22D0102004F0ECFE90
:10690000041E1DD01022002104F0E6FD2620FFF712
:1069100059FC002800D13078D0232370C13BA370EC
:10692000009B21002372019B67706372029BA5800C
:10693000A372039BC0B2E3720C9BE36004F08CFE75
:1069400005B0F0BDF7B50D00019001F033FE071E54
:1069500020D00E2004F0C0FE041E1BD02620FFF71E
:1069600031FC061E00D13E78D0232380C53B062291
:10697000A370F91DE01C04F08FFD019B2A006381C8
:106980000123DD401A401D40210022736573F0B2DF
:1069900004F062FEF7BD0000F0B585B00290100073
:1069A0000D0017000A9E039301F004FE041E31D06F
:1069B000029B002B2ED1039B02795B0724D5122367
:1069C00013430422002E08D10B99002905D10C99FC
:1069D000002902D10D9900291AD01A430D9B22716A
:1069E000002B00D0C9E0002E00D1CFE0002D00D058
:1069F000CCE0606A002801D004F046FD1C21300084
:106A000004F07AFE606205E002239A430E33D7E772
:106A100093432371654BBA00D458002C00D1AAE0EF
:106A2000002E10D0236A002B03D11C2004F07CFD23
:106A300020625E4BBA00D358186A002803D01C228B
:106A4000310004F029FD0C9B002B12D0574CBB00E9
:106A50001D596B6A002B03D1162004F065FD686296
:106A6000BB00E358586A002803D016220C9904F0A2
:106A700013FD0D9B002B11D04C4DBC006659B36A21
:106A8000002B03D1142004F04FFDB0622B59986AFB
:106A9000002803D014220D9904F0FEFC380001F008
:106AA00089FD051E67D0414BBA00D358002B62D038
:106AB0001A6A3420002A00D11C389A6A002A01D0B0
:106AC000143080B20B9A002A01D01C3080B25B6A6D
:106AD000002B01D0163080B204F0FEFD041E4AD017
:106AE0001822002104F0F8FC2620FFF76BFB019030
:106AF000002801D12B780193D0232370029B200022
:106B000063700A23294EA370039BBD00A371AB5988
:106B1000A780196A1830002905D01C22A06004F053
:106B2000BBFC200034307359996A002907D0030058
:106B300014221433E060029304F0AEFC02980B9B25
:106B4000002B08D003001C221C330B9920610293F8
:106B500004F0A2FC02987359596A002903D0162246
:106B6000606104F099FC6B462100187904F074FD13
:106B70003800FFF7E3FC05B0F0BD10220D9B0D9926
:106B80001B69A018236204F087FC2CE70B9B002BE9
:106B900000D13FE7012D00D03CE7606A002801D01A
:106BA00004F072FC1C210B982AE7C046AC66FF1F5C
:106BB00010B5044C2068002803D004F065FC0023C5
:106BC000236010BDA066FF1F0B4B07B51A68002A93
:106BD00001D100200EBD6946531C012012780731F7
:106BE000FFF772FC0028F4D002780123100018404F
:106BF0001A42EED0EEE7C046BC66FF1FF0B51F4F4D
:106C000001203B6887B0002B25D09B78059300F0CE
:106C1000B3FB002821D00A20FFF7D4FA04000B2090
:106C2000FFF7D0FA164B05001E78731E9E413B6895
:106C3000F6B2191DD878FFF757FB3B682900DA7ABE
:106C4000043303929A79019302920090330020005A
:106C5000059A04F0D1FD07B0F0BDFFF7B5FF00289D
:106C600005D00620FFF7AEFA04000720D8E7082079
:106C7000FFF7A8FA04000920D2E7C046A066FF1F6C
:106C80009C66FF1F70B50A4E040033780D00FF2B81
:106C90000DD0042004F020FD011E08D0D023037085
:106CA000CE3B45708370C470307804F0D5FC70BD65
:106CB0002045FF1F70B5040006200D0004F00CFDF8
:106CC000011E0AD0D0230370CD3B8370054B447066
:106CD0001B688580187804F0BFFC002C01D0FFF7FA
:106CE00067FF70BDA066FF1FF8B5264F06003B6822
:106CF0000D001124002B05D10522234B1B781342D4
:106D000002D112242000F8BD204A10241268002A63
:106D1000F8D01278002AF5D0DB0719D52B789A1E07
:106D2000012A1AD80C2004F0FFFB13243860002835
:106D3000E8D000230A22437029000670023004F0D4
:106D4000ABFBFFF75BFF041E0AD0FFF731FFD9E76B
:106D500000F012FB0028E1D1E4E7002BE2D0D0E7FD
:106D60000B4B1B78032BCDD11D20FFF72BFA094BC2
:106D700018800028C6D0084B04211878074A04F070
:106D80007BFBBFE7A066FF1F9D66FF1FBC66FF1F62
:106D90009C66FF1F9A66FF1FC866FF1F60EA00001F
:106DA000F7B50193194B14001A78052306000F005C
:106DB00012201A4221D0012920D1154B1D68002D27
:106DC0001BD002201F2C18D8002C02D0019B002BB6
:106DD00013D0104B1F221E706E1C0021300004F0D7
:106DE0007BFB01992200300004F056FB31002000AB
:106DF0002C70002F06D004F067FAFEBD064B12205F
:106E00001D68DCE704F0F8FBF7E7C0469D66FF1F4E
:106E1000BC66FF1F2045FF1FB866FF1FF8B50F4E69
:106E200012243368002B17D01B780F3C834213D1F8
:106E300000250B4F0221387804F07EFB094B04211A
:106E400038781D8004F078FB074B28001D803368DC
:106E50005C7004F0B1FA04002000F8BDA066FF1FCA
:106E6000C866FF1FB466FF1F9A66FF1F70B5012832
:106E700023D11B4C2388002B03D01A4A1578002DF0
:106E800007D0194B1B68002B02D01878FFF7C6FFFC
:106E900070BD3B2B02D93C3B2380F9E7134E022106
:106EA000307804F049FBFA222388920002215A43E9
:106EB000307804F029FA2580EAE70B4B1B68002B99
:106EC000E6D00B4B1B785B07E2D5084B0221187804
:106ED00004F032FB0022024B1A80FFF769FED7E76D
:106EE000B466FF1F9866FF1FA066FF1FC866FF1FDE
:106EF0009D66FF1FF8B51E4D2868002803D004F0DA
:106F0000C3FA00232B601B4E3068002803D004F026
:106F1000BBFA00233360184F05243B78180020404B
:106F2000234221D0154800F02BFA3B78234213D09E
:106F3000202004F0F9FA2860002813D02022002134
:106F400004F0CAFA202004F0EFFA041E306005D0E5
:106F50002022002104F0C0FA002004E0286804F098
:106F600093FA2C601320F8BD00F00AFAF4E7C0464B
:106F7000BC66FF1FB866FF1F9D66FF1F1445FF1FFD
:106F800010B50A4C23681A1E0ED0002808D1013013
:106F9000587004F011FA002805D02368002B02D0A5
:106FA0000021FFF787FE0122100010BDA066FF1F21
:106FB000F7B5274E050033680191181E21D05C7883
:106FC000244F012C30D1FFF7FFFD002825D02000F1
:106FD000FFF7F8F80400412814D91F4B0221187854
:106FE0001E4A04F049FA1E4B3C3C1C8002223368C6
:106FF0005A703B78002B14D128000199FFF75AFEF4
:107000000120FEBDFA2292004243002AEED0124B2C
:107010000221187804F078F9E8E7FFF7D3F80200C6
:10702000F3E700233B70EBE73B78002BE8D103202C
:1070300004F052FB011E08D0D0230370CC3B4570F6
:1070400083703368187804F007FBFFF7B1FDD7E7CA
:10705000A066FF1F9866FF1FC866FF1F60EA00005A
:10706000B466FF1F10B51749838802008B4220D0F9
:1070700011D815498B4217D0144900205B1899B2DA
:10708000012907D8926811785A425341D8B2FFF7C4
:10709000F9FD012010BD0E4A00209B1807229BB26B
:1070A0009A424041C0B2F5E783681878FFF768FF5D
:1070B000F0E7836899785A78090218781143FFF746
:1070C00077FFE7E70A20000006200000F8DFFFFF57
:1070D000AFDFFFFF014B18707047C0462145FF1F0F
:1070E00010B5064C207001F041FA207804F0CCFB7A
:1070F0000521207800F062FD10BDC046C866FF1F64
:107100000BB273B50D00002B00DBC4E0884B187880
:1071100004F072F9041E0ED00378912B0FD0A22B2D
:1071200000D1A1E0834B1878FF2852D0210004F051
:1071300093FA00284DD180200002684076BD437844
:107140000F2B76D013D8052B70D00E2BEAD1808868
:10715000794B98422BD8794B98421BD8784B984260
:10716000E0D1A3681878591CFFF774F838E03E2B7B
:10717000D8D18378032B74D06CD8012B6ED0022B1E
:10718000D0D1704B1B68002B23D05B68002B20D024
:1071900098471EE06C4BC0180C28C3D804F0E4F8E4
:1071A0001DC2C2150BC20B0B0B3223C23C00674B36
:1071B000C0180728B6D8664B1B68002B09D01B687F
:1071C000002B06D0200098470AE0A3681878FFF744
:1071D000C7F8200004F0A8FAADE7A068FFF762F84E
:1071E00000289FD0F5E7A3681B78002BF1D0554B02
:1071F0001B68002BEDD01B68002BEAD021005548FE
:107200009847EDE74F4B1B68002BE2D01B68002B23
:10721000DFD021005048F3E7504B1B68002BD8D03B
:107220005B68002BD5D021004348E9E7FFF7EAF976
:10723000CFE780884A4B984203D04A4B984200D00F
:1072400070E7464B1B68002BC3D05B68002BC0D097
:107250002100D5E7153B012BBBD963E7FFF798FA6F
:10726000B7E7FFF77DFAB4E73F4B1B78042B07D154
:1072700000236A4613800179408800F0C5FCA8E726
:10728000364B1B68002BA4D05B68002BA1D00100FB
:10729000364898479DE7012421420AD0294B1B68B4
:1072A000002B04D05B68002B01D000209847012000
:1072B00043E78B070AD5264B1B68002B04D05B687D
:1072C000002B01D020009847022036E70421280037
:1072D00008400D4200D131E7254E3388002B21D0E4
:1072E000013B9BB23380002B1AD1FFF7DBF800285B
:1072F0000AD0204B1C70164B1B68002B04D05B6817
:10730000002B01D020009847FFF7C6F8694601F02E
:1073100001FD6846FEF7FEFF1D20FEF753FF30809B
:1073200004200AE7024B187804F006F9F8E7C04693
:10733000C866FF1F2145FF1F0E200000012000002E
:1073400009100000C066FF1FFEDFFFFFAFDFFFFF79
:10735000C466FF1F0C2000000B200000A866FF1F62
:107360000D200000132000009D66FF1FFFFF00009E
:107370009A66FF1F9866FF1F10B501F09BF910BDBC
:10738000014B18607047C046C466FF1F0B88002081
:10739000162B01D817230420014A13807047C046DA
:1073A0007266FF1F00207047074A03001188814260
:1073B00007D091880020994202D101308000101836
:1073C00070470020FAE7C046D066FF1FF0B58F78FF
:1073D00006000D00C7B01E2F15D1FFF7E5FF051EF3
:1073E00003D10024200047B0F0BD00223B00310053
:1073F000C078009200F0B2FB0400A81C00F0D3FBA0
:10740000FF23EB70EEE7264B062403931B78FF2B3C
:10741000E8D0182FE6D87B08224A013BDB00029215
:107420009A589446002ADDD0029AD3185B68002B44
:10743000D8D00878002802D14B78012B02D106243D
:10744000122FCFD107AFAB88697800976446AA683E
:10745000A047041EC6D1AB78029A5B08013BDB0053
:10746000D318390030005B689847041E0BD1AB7805
:10747000042BB6D0039A310010782200009700F058
:107480006DFB0400AEE76A78002AABD1AA7805A9A3
:107490003B88087130000A704B80FEF747FBA0E77D
:1074A0002445FF1F64BB00111D4B37B505009842F2
:1074B0000BD000290AD1FFF777FF002805D1194822
:1074C000FFF772FF002800D0058037BD01291AD1CF
:1074D000FFF76AFF041EF8D001235B420380A37804
:1074E000FF2BF2D0FE2B07D00023E078142200936C
:1074F00029001E3300F032FBA01C00F054FB0123D6
:107500005B426380E1E70229DFD1013901F0BEF877
:107510000028DAD12800FFF747FF041EDFD1D4E7A7
:10752000FEFF0000FFFF0000022210B5074B524291
:107530001A80074801325A809A80DA8000F07EFA79
:10754000044801F025F8002010BDC046D066FF1F9A
:10755000CD730011A97400110388F7B50400002B46
:1075600002D102252800FEBD426802211378254879
:107570005268FEF7A5FD00282ED0234F01253A883A
:10758000002AEFD0802321885B0201259B1A9942B3
:10759000E8DC0C2003F0C8FF061E31D03B882288AF
:1075A0009C4600231800019561469DB2491989B295
:1075B000AA421BD8002801D062443A800023300040
:1075C000082208C0210003F067FF104A1368002B4F
:1075D00013D100251660C5E76268022113780C48B4
:1075E0005268FEF76DFD0028C7D1BAE760681D013B
:1075F0004019418101330198D6E71A001B68E6E77C
:107600001325AFE7D2BB00112245FF1FCC66FF1F39
:10761000D0BB0011014B18707047C0462445FF1FB6
:1076200014230A0010B51A40194204D00122102177
:1076300001F048F810BD4B06F9D401208843400002
:10764000F8E710B514008B0604D50122102101F0D3
:1076500039F810BD08230A001A40194202D14BB272
:10766000002B0FDA102101F02DF8002808D023009C
:10767000F9331B78002BECD0F8342378012BE8D1B8
:107680000020E6E703208907FAD4E2E7F0B51F00FF
:10769000184B85B01C68019002910392002C27D1F1
:1076A000200005B0F0BDA5683301ED186B89019A83
:1076B000934211D3029A93420ED8002F04D10A9B11
:1076C000002B10D12C00EBE73B002978039A686867
:1076D000FEF7F6FC0028F2D10136B6B2A388B34219
:1076E000E1D82468DAE7A3680A9A5B891380E9E79E
:1076F0000026F3E7CC66FF1F37B50C000A884988DF
:107700000123914217D3002A15D0651D23792A0041
:1077100002210A48FEF7D4FC102300280BD023795D
:107720006188208800242A000094FFF7AFFF0A2315
:10773000A04200D0230018003EBDC046D2BB0011BD
:1077400013B50A0008884988012388420BD800280D
:1077500009D00024137905320094FFF797FF0A231C
:10776000A04200D02300180016BD13B50A000888F7
:107770004988012388420BD8002809D000241379B6
:1077800005320094FFF782FF0A23A04200D02300B5
:10779000180016BDF0B58BB003904A8808880E001B
:1077A0000123824255D3002853D00023012704AC83
:1077B00023700022718813000092FFF767FF051EF7
:1077C0003ED02078002835D12B78022B18D1677055
:1077D0006A8983000130E31880005A8069680222B8
:1077E000201803F059FE23780133DBB22370042BF9
:1077F00019D93B006889013080B2002BD9D01FE035
:1078000002236370122358436A89231804305A8074
:1078100069681022201803F03FFE23780133DBB2A1
:107820002370002BE5D10C4A6B899B185A425341B7
:10783000DBB2DFE76378012BE4D12B78022BC7D0D2
:1078400022780A23002A04D021000398FEF798F931
:10785000002318000BB0F0BD0100FFFF0F4BF0B587
:1078600004001868002816D083685D89A54207D8EF
:107870008288AE18B44203DA12019A18934201D1F9
:107880000068EFE71E005F891036A74204D1002987
:1078900000D00D801800F0BD3300EFE7CC66FF1F6D
:1078A00070B505000C0008880021FFF7D7FF030022
:1078B0000120002B04D022002800197AFFF7C1FE16
:1078C00070BDF7B50C00002501902300F6331B783E
:1078D000AB4201D800200AE06B00E65A00213000DC
:1078E000E718FFF7BBFF002802D126800130FEBD5C
:1078F000017A0198FFF794FE002802D03B8823808C
:10790000F5E70135EDB2E0E710B504000888002185
:10791000FFF7A4FF03000120002B03D02000197AF9
:10792000FFF77EFE10BD0000054B1B68002B01D148
:10793000180004E09A6852898242F6D1988870470C
:10794000CC66FF1FF0B50E27002687B0039302AB6D
:10795000FF183E8005001F4B40891400984207D055
:107960002B78013000976A6880B2FFF78FFE06001F
:1079700002212B7818486A68FEF7A2FB00280FD076
:107980006C892000FFF7D0FF002802D0013C0419C9
:10799000A4B2039B002B00D01C80300007B0F0BDC8
:1079A00002212B780D486A68FEF78AFB0028E7D190
:1079B00002212B780A486A68FEF782FB002807D06C
:1079C000002EDED03B88A342DBD17489013CDFE787
:1079D0006C89DEE7FFFF0000D2BB0011D0BB0011B5
:1079E000CEBB001110B50C00FFF7DEFC0300022037
:1079F000002B0AD0002C00D023609B781720FE2B90
:107A000003D00138FF2B00D1002010BD73B50D004D
:107A100001A904001600FFF7E5FF172805D0002E86
:107A200004D129002000FEF727F976BD012210219C
:107A3000200000F047FE0028F3D0F6E7014B186065
:107A40007047C046DC66FF1F37B56B469D1D0100C1
:107A500004000222280003F09FFC2B88B02B0ED1DB
:107A60002379122B09D12300FF339B78012B06D1F8
:107A70000121608800F0E0F801E01B2BF8D037BD51
:107A800010B5054B0421187000F098F8FFF74CFD75
:107A9000FEF770FB10BDC046E066FF1F0020F0B58A
:107AA0000BB20F0087B0834234DA274B187803F00B
:107AB000A3FC051E2BD00378A02B25D103AE3100EB
:107AC000FEF7E4F8041E0BD1B378DB0724D51F4B77
:107AD00006341B68002B03D03100688898470400E7
:107AE000A868002801D003F0F7FB002C08D1184A41
:107AF000039B1340174A934206D0B3781B2B03D045
:107B00000121688800F098F8280003F00DFE80201D
:107B10000002784007B0F0BD0F4B1B68002B10D05F
:107B2000310068889847041EDAD07378002BD7D1CB
:107B3000B27801A90A704B800C716888FDF7F6FFD6
:107B4000CEE70624F1E7C046E066FF1FD866FF1FB8
:107B500000FFFF0000011200DC66FF1FF7B5019077
:107B6000822040000D0017001E0003F0B5FD040048
:107B70001320002C12D0B02320002370089BFC227D
:107B80006770658026710830002B08D0190003F05B
:107B900083FC2100019803F05FFD0020FEBD0899E1
:107BA00003F09AFCF5E710B5041E06D00078FD2816
:107BB00003D803F0C9FDFF23237010BD0A1F93B241
:107BC00010B504000220032B05D882400020024B90
:107BD000D1529B189C7010BD0067FF1F0B8870B5B9
:107BE000043B04000D000220032B0BD801212000D0
:107BF00000F04CFD03001420002B03D029002000CE
:107C000000F0DEFB70BD000007B51300034A0092D0
:107C10000A00012100F02CFC0EBDC046457E00117B
:107C200007B5019203220092024B0A00122100F0D4
:107C300049FC0EBDC37E001107B56B4601AA118039
:107C40000449D88008780633012802D1190003F0CE
:107C500063FE07BDE166FF1F0C4B10B518700023D3
:107C6000FF210B4A1380138193819380094A53802B
:107C70001370517293819372D174D38213755177BB
:107C800003F0D2FB00F0FCF910BDC0461067FF1FE7
:107C90000067FF1FE266FF1FF0B58DB06B46002046
:107CA00003910C229B5E834200DBB0E05D4B1878B1
:107CB00003F0A2FB051E00D1A4E00378902B00D0B6
:107CC0009DE006AF01004688380000F013FA79689D
:107CD0000400002900D19CE03B88052B6ED13B8934
:107CE000032B1CD905AC200000F0A2F86288172AEB
:107CF00061D83989131D994231D1796823780431CB
:107D00000291D90738D5607800F08EF9071E06D0A9
:107D1000002303712378012B08D0132B23D0A868EC
:107D2000002800D178E003F0D7FA75E06288029964
:107D300009A800F0A6F80290380000F08BF909AA13
:107D40002378387A0192002231000092029A00F0E2
:107D500012F9380000F064F9029B002BDFD03000EC
:107D600000F080F9DBE70378032BD8D16288029911
:107D700009A800F0D6F8DEE7122B13D1029909A862
:107D800000F0B5F8021EEAD127498B88002BC6D037
:107D9000887909A92378019161780091310000F078
:107DA000EAF8BCE7002302AA93833000617809AAAD
:107DB000FFF72AFFB3E71D4B0993F6E7042B02D028
:107DC0009A1F012AABD8184A043B9B00995A0029F4
:107DD000A5D0D218907831003A0000F0AEF8002813
:107DE0009DD13B88042B03D001213000FFF724FFF5
:107DF000012C04D1A868002801D003F06DFA2800F6
:107E000003F092FC8020039B0002434018000DB059
:107E1000F0BD012800D182E701213000FFF70CFFFF
:107E2000EDE7C0461067FF1F0067FF1F0100170046
:107E30000B7803704B784370CB788A781B0213431E
:107E4000438070470A88030002700A88120A427051
:107E50000A88012A06D14A8882704A88120AC270AA
:107E60000420704702208242FBD14A8804309A7075
:107E70004A88120ADA708A881A718A88120A5A7134
:107E8000EFE710B50400012082420CD94B780A7844
:107E90001B0213432380834206D1CB788A781B02CE
:107EA00013436380002010BD022BFBD1CB788A786E
:107EB0001B02134363804B790A791B021343A3808F
:107EC000F0E70B8803700B881B0A43704B888370A4
:107ED0004B881B0AC3708B8803718B881B0A437104
:107EE000CB888371CB881B0AC371082070470300BD
:107EF0000120082A14D14A780878120202431A8015
:107F0000CA788878120202435A804A7908791202A4
:107F100002439A80CA798879120202430020DA80EB
:107F2000704710B504000120022A05D100204B78CB
:107F30000A781B021343238010BDF8B506001020F9
:107F40000F00150003F0C8FB04000120002C0ED028
:107F5000A0230C22290023806780201D002D07D03C
:107F600003F09AFA2100300003F076FB0020F8BD00
:107F700003F0B2FAF6E7F7B51E00009008AB142044
:107F800017001D78019103F0A7FB041E12D0A22355
:107F90000370019B47704380099B057146710C2259
:107FA0000830002B07D0190003F076FA2100009862
:107FB00003F052FBF7BD099903F08EFAF6E737B5E7
:107FC000041E0FD04388002B0CD00025C18813233A
:107FD000007A172201950095FFF7CDFFFF236580FA
:107FE0006372257037BD000010B50C4904004A8843
:107FF000002A09D08B89002B05D00020CB8A0222D1
:10800000834201D010BD012213000A204343002007
:108010004032C854C81842800472F3E7E266FF1F7A
:108020000023438003707047094B00211A0010B5EC
:108030005C88002C06D01C79844203D10A234B4370
:10804000D01810BD01310A330329F1D10020F8E71F
:10805000E266FF1F10B50400407A03F075FBFF23B2
:10806000637210BD7047043010B580B203F014FB8A
:10807000002803D00421494203F0DEFB10BD0000BC
:1080800070B50025104CA0682580A581A580A84268
:1080900002D003F021F9A56000250C4C0C4B606D5B
:1080A0001D80230058331D70A84202D003F014F93C
:1080B000656500256068002801D003F00DF90135E1
:1080C00008340A2DF6D170BDA867FF1F4C67FF1F4B
:1080D0009C67FF1F70B5041E09D1054D2880A8813B
:1080E000A880A868002802D003F0F6F8AC6070BD44
:1080F000A867FF1FF0B54B8885B00193002343604C
:108100000A7905000F00022A00D07BE0CA88032A02
:1081100017D98B685E7819783602DC78D8790E43E7
:1081200099781B7A24021B020C43034353495BBA20
:108130000B80331D93421ED1042C04D0631F022BED
:108140000ED9012015E0019A4D4B1201D35A002B94
:1081500006D00198FFF7BEFF4A4A13690133136145
:108160000421B8682E812C80494203F065FB6860C9
:10817000002005B0F0BD434D042C06D0631F022B38
:108180000FD9EB680133EB60DBE7019A3C4B12013E
:10819000D35A002B05D00198FFF79CFF2B690133C0
:1081A0002B61374B30000293019B029A1B01019314
:1081B000002301998C468B52130063449C800393E7
:1081C0009E81FFF750FF039B041E986016D0042188
:1081D000B868494203F030FBFA880100043A2000F5
:1081E00003F05AF90199029AFB888A5A043B9B18BA
:1081F000029A8B522B6801332B60A2E7AB690133E3
:10820000AB619EE71E4B0293019B1E01029BF35A3A
:10821000002B2DD002998C19A068002828D0012AA3
:1082200026D1FA889B189BB27352A189994217D321
:108230009B1AC018B96803F02FF9029BA289F35A60
:10824000934200D07DE700222B81A3882B80A36876
:108250006B60029BF2520B4A53680133536070E724
:10826000084A9368013393600198FFF733FF68E78A
:10827000044A536901335361F6E7C0461267FF1F92
:10828000A867FF1F1867FF1F70B5051E15D10B4C9F
:108290000B4B1880230058331870606D002802D0F3
:1082A00003F01AF86565250050356068002801D094
:1082B00003F012F80834AC42F7D170BD4C67FF1FD1
:1082C0009C67FF1FF0B51700A12285B092000193B3
:1082D0004243394B06001B680C009B18D933FF330F
:1082E0001D78FDF741FF0430854204DD3000FDF7C5
:1082F0003BFF0430C5B2BD4207D33A000021300035
:10830000019B03F069F805B0F0BD2900380003F0C7
:108310009BF82300C6B250331E700393019B2900C3
:108320006365380003F018FBCBB20293002B02D038
:10833000039B01361E7000262300503303931B78E5
:10834000B34204D8606D002831D10020DBE7029AE7
:108350002800002A04D0013B1000B34200D02800BE
:10836000F700E719387002F0E7FF786000280ED0B8
:108370003A78019903F090F8019A3B780136D318C6
:108380000E4A0193D369F6B20133D361D4E7039B5C
:1083900018706065A74205D1084A1320D36A0133DB
:1083A000D362B0E7606802F097FF0834F2E702F0AA
:1083B00093FF00236365C8E73409FF1F1867FF1F99
:1083C000F7B50D0007000421686803F035FA2B8922
:1083D000040003702B891B0A43702B8883702B8841
:1083E0001B0AC3702E8902250436F6B2FB2E15D85F
:1083F0001B4B9F4214D10C2003F06EF91135011E66
:108400000CD0902303708E3B0371043B4380154BCB
:108410008460C680187803F01FF900252800FEBD8F
:108420005C237B43104AD3180093583301931B7885
:10843000002B0FD10300320038000099FFF742FFF4
:10844000019B05001B78002BE8D13800009903F050
:10845000FBF9E3E7054A0725536A01335362DDE779
:10846000FEFF00001067FF1F4C67FF1F1867FF1F0C
:10847000F0B587B0009017200F0016000193FFF7AA
:10848000F2FD1325041E19D00C98031E02D0019989
:10849000201D9847030AE370052302AAA070043048
:1084A000908127700098667003A993800494FFF769
:1084B00087FF051E02D0200002F00EFF280007B043
:1084C000F0BD0000F0B587B01F000CAB1B78039126
:1084D000059301210DAB06001C78049200F0D6F83C
:1084E0001425002821D02000FFF77EFD0135041E51
:1084F0001BD01149059B0A7803700132D2B2131EBA
:10850000C68001D101231A000B7022713000049B38
:1085100003990097FFF7ACFF051E09D12300210046
:108520000648074A093303F0A7F8280007B0F0BD52
:10853000002363802370F8E71467FF1FBF7F0011DB
:1085400030750000F8B505000E00064C064F236894
:10855000002B02D03100280098470434BC42F6D1E9
:10856000F8BDC046B867FF1FCC67FF1F0123064A4E
:108570005B425380002313715362044A13605360BB
:108580009360D36013617047CC67FF1FB867FF1F0C
:108590000200002310B506499C000859002801D1AB
:1085A000625010BD0133052BF6D11320F9E7C04608
:1085B000B867FF1F034A5388181A43425841404284
:1085C00010407047CC67FF1FF0B585B002930AAB2F
:1085D0001F780CAB1B88009008000E0001920393DB
:1085E000FFF7E8FF05001120002D1BD10E48FFF713
:1085F000E1FF04001520002C14D006220B99A7716E
:10860000E01D02F049FF019B30002371029B29000D
:108610006371009B66802370039B6562E381FFF7B3
:1086200091FF280005B0F0BDFFFF000010B5FFF777
:10863000C1FF04000220002C12D060880121FFF746
:1086400081FF606A002801D002F01EFF282200216D
:10865000200002F041FF012300205B426380207173
:1086600010BD000030B5074A074C5588010013784B
:108670000020A54204D05B1A59424B415842104099
:1086800030BDC046CC67FF1FFFFF0000084A10B591
:1086900001230C00904208D0FFF78CFF031E04D08A
:1086A000037923405A1E9341DBB2180010BDC04627
:1086B000FEFF0000024B1879431E9841C0B270477C
:1086C000CC67FF1F70B504000D001600FFF772FFA6
:1086D000002804D10D4B9C4200D0143070BD416A7B
:1086E00003790520002907D012221A40102A02D14E
:1086F0000520002EF2D10F20DB06EFD5897E0C205D
:10870000A9428941494249420840E7E7FEFF00008B
:10871000030010B5002800D110BD0348034A41886A
:108720009142F9D09847F7E7CC67FF1FFFFF0000A1
:10873000002330B5C45CCD5C6C40D4540133102BA5
:10874000F8D130BD0F23002210B5C45C6400224371
:10875000CA54C25CD209013BF7D210BD020001002D
:1087600010B52032103103F097F810BDF0B58BB082
:108770000390102005931700049102F0D5FE00909D
:10878000102002F0D1FE009B13240190002B05D095
:1087900000280CD11324009802F076FE019B002BD8
:1087A00002D0180002F070FE20000BB0F0BD1020C7
:1087B00002F0BAFE0600102002F0B6FE13240500F7
:1087C000002E00D1AEE0002819D01022002102F0C6
:1087D00083FE32002900039803F05EF8041E0ED1D8
:1087E00033787F2B51D830000099FFF7ABFF009B07
:1087F0001B787F2B53D801990098FFF7A3FF300017
:1088000002F042FE002D02D0280002F03DFE002CB6
:10881000C1D1102002F088FE0600102002F084FE74
:108820000290002E7CD0002878D03A000F3223002E
:108830000125121105D00F333B4015B25A42534166
:108840001BB26A1E1201002B33D0049BD2B29818BF
:108850000099029AFFF76CFF013D102200213000C1
:1088600002F03AFEADB2049F2D017D19AF4242D015
:10887000002C33D0300002F007FE029B002B00D109
:1088800089E7180002F000FE85E729003000FFF7B5
:1088900059FF28002549009AFFF74AFFA7E729005A
:1088A0000098FFF74FFF28002049019AFFF740FF8B
:1088B000A5E70F210F4004998A18D9B28F4208D931
:1088C000D15C06A819540133102BF6D1029A0199F4
:1088D000C0E7791A48424141C901F2E73900300046
:1088E00006AAFFF725FF3200039806A902F0D4FF7D
:1088F00010370400BAE7002CBCD13000029906AA58
:10890000FFF716FF320006A9039802F0C5FF082200
:1089100004003100059802F0BFFDABE71324A9E77E
:108920001324AAE7002800D06EE733E7D8BB001174
:10893000F0B58BB00F0016000225009000283FD044
:10894000002A3DD00B1DDBB21800029302F0ECFDB3
:108950001135041E34D0FDF747FD05003A0000999B
:10896000201D02F039FFEBB20393E3702B0CDBB256
:108970002F0A00936370FFB22B0E2370A770019330
:10898000FDF72CFD1022010006A802F025FF2100B2
:10899000029A04AB06A8FFF7E9FE051E0DD1039B62
:1089A00008223370009B04A9B370019B7770F370A9
:1089B000301D02F011FFFDF71DFD200002F064FDE7
:1089C00028000BB0F0BDF0B58FB00D00149E0390E1
:1089D00004920593002A03D1022420000FB0F0BDB9
:1089E000002EF9D00398FFF7E5FD1424071EF4D0FC
:1089F0007278337812021A43B3781B041343F27867
:108A000012061A43036A0192934201D30133E3D160
:108A1000002D03D03B7901249B07DED508220021DD
:108A200006A802F059FD059B13240433DBB218009D
:108A3000029302F079FD051ECFD0059A0499043007
:108A400002F0CAFE04223100280002F0C5FE3900FF
:108A5000102210310AA802F0BFFE2900029A06ABCC
:108A60000AA8FFF783FE041E0FD1082206A908A852
:108A700002F0B2FE0822311D08A802F0E5FD01282F
:108A800007D101990398FDF7C9FC280002F0FCFC0E
:108A9000A3E70124F9E7000070B51C4C050023682A
:108AA000181E10D0002D14D11A78002A0CD1981C51
:108AB000083202F0F1FC02F0AFFD0135002808D1C8
:108AC00023681D70012070BD0A331800082202F0CF
:108AD000E3FC2368002BF5D0122002F0FDFD061EFA
:108AE0000DD0C1232168037045700231102202307D
:108AF00002F0D2FC23683100587802F0ADFD206806
:108B000002F0C2FC00232360DCE7C046F467FF1FCD
:108B1000F8B504002020FDF755FB0D4EA700BB590A
:108B20000500002B0DD000280BD0D878FF2809D1E4
:108B300008492A000C55F35907480333611802F01D
:108B40009BFDF8BD290002F02FFE0028F0D1F8E7C8
:108B50001068FF1FF867FF1F699D001170B5064D73
:108B600084006359002B05D0D87802F0EDFDFF2278
:108B70006359DA7070BDC0461068FF1F70B50600FB
:108B80008CB00C00150000213022684602F0A4FCD5
:108B900031001022684602F01FFE1D202100032232
:108BA000684402F019FE6846FFF7D8FD2D21040045
:108BB00003222800694402F00FFE20000CB070BDB3
:108BC000F0B50700160097B001931CAB1D7830225A
:108BD0001EAB00910AA800211C7802F07DFC102237
:108BE00039000AA802F0F8FD1022002102A802F0C4
:108BF00073FC0722310002A802F0EEFD072202AB4F
:108C00009818631E9C41019902F0E6FD02AB9C732B
:108C10002B005A1E934102AAD3730021102206A8EA
:108C200002F05AFC06221D9907A802F0D5FD1A2071
:108C300002ABC01806221F9902F0CEFD1022009947
:108C40000EA802F0C9FD102202AB0EA908781C780C
:108C5000013A6040D2B2087001330131002AF5D1E7
:108C60000AA8FFF77BFD102212A904000EA802F04B
:108C700013FC102206AB0EA908781D78013A684053
:108C8000D2B2087001330131002AF5D10AA8FFF7EA
:108C900065FD044310222098E4B212A902F09CFD65
:108CA000200017B0F0BD70B50E0014008CB00100AC
:108CB000102268461D0002F08FFD3100082204A832
:108CC00002F08AFD2100082206A802F085FD684610
:108CD000FFF744FD04001022280008A902F07CFDE3
:108CE00020000CB070BDF8B506000D000024371947
:108CF000AC4200D3F8BD02F0B7FD030A3B70631C21
:108D0000DBB201379D4203D90234F054E4B2EEE7FE
:108D10001C00EDE773B506000C000225002819D0F1
:108D2000002917D0032101A8FFF7DDFF6B469A79D0
:108D30003F231A40013313436A463000937101A95F
:108D40002200FFF71BFF051E04D10322E01C01A92E
:108D500002F0A2FB280076BD03785807DA08C00F9E
:108D6000D20080009B0710439B0F1843C0B270478E
:108D700007230B40C908C9000B430370704700006C
:108D800070B50400FFF7EAFE134DA4006359002BF1
:108D900021D0186A002801D002F076FB2B59986E7A
:108DA000002801D002F070FB2B59D86E002801D0AA
:108DB00002F06AFB2B59186F002801D002F064FB07
:108DC0002B59586F002801D002F05EFB285902F0A1
:108DD0005BFB00232B5170BD1068FF1F0E4B800002
:108DE000C35870B50C00002B0FD09D68002D0CD01F
:108DF0002B78201D0B706B784B70A97CFFF7B8FFA8
:108E00002B7E23726B69E36070BD1022002120006D
:108E100002F062FBF8E7C0461068FF1F014B1860C4
:108E20007047C0460C68FF1F074A03008000825845
:108E300010B5002A06D0D088984203D1012901D16B
:108E4000FFF79EFF10BDC0461068FF1FF0B5264E0D
:108E500095B087000B93BB590500099112200A9227
:108E6000002B31D0D888FFF7A5FB04001420002C7C
:108E70002AD0280010A9FFF7B1FFBB591E781D6A40
:108E8000002E23D00895FDF7EFFA07000020FDF72C
:108E9000F1FA0790A379E61D069310AD0CA9089886
:108EA00000F0E2FA0EA9280000F0D7FA0B9B0A990D
:108EB0000493069B09980293079B039601930097DE
:108EC0000EAB0CAAFFF77CFE15B0F0BDFDF7CCFA97
:108ED00006903000FDF7CEFAE31DA779079310AB9B
:108EE00006000893DAE7C0461068FF1F30B50C4C47
:108EF00085002A59030085B00120002A0ED01800F1
:108F00006946FFF76BFF2B591A78D888054B002A62
:108F100000D1054B6A46072100F0D9FB05B030BDF2
:108F20001068FF1F5B9400116994001130B5094C63
:108F30008500295985B010226846253102F0ACFA27
:108F40002A591121044BD0886A4600F0C0FB05B0B5
:108F500030BDC0461068FF1F0595001130B5094CA3
:108F60008500295985B010226846353102F094FAFF
:108F70002A591121044BD0886A4600F0A8FB05B09D
:108F800030BDC0461068FF1F43950011F7B54D4F27
:108F900086001020F4590D0002F0C6FAF359206241
:108FA000186A132200286CD0033A29009C6802F04A
:108FB00073FAF3591A780192002A58D11E6A227D59
:108FC000317B944651400122019F114201D16746F5
:108FD0001740217D914339432175377B4F40BC4673
:108FE00060460027800701D44F0817400121022066
:108FF0008F40227D82433A432275377B5740BC46DF
:1090000060460027400701D497080F400420227DC6
:10901000BF0082433A432275627D00279446604632
:10902000727B42400A4201D167460F400121627DB6
:109030008A433A436275777B5740BC4660460027B7
:10904000800701D457080F400220627D7F008243D1
:1090500017436775767B00227E40760701D4BA08F5
:109060000A400426617D9200B1430A4362756A7822
:10907000002A08D06278002A05D005220533DA7765
:1090800000221000FEBD04222979114205D1A17CE5
:10909000114202D10533033AF1E7019A21782C7885
:1090A000002A02D10A002100140018220429E8D85D
:1090B000042CE6D805206043034A05331218525C9D
:1090C000DDE7C0461068FF1FE8BB001110B50A00BD
:1090D0001121024B00F0FBFA10BDC0469F95001114
:1090E0000B0030B587B001AD2B806B46040011003A
:1090F000981D082202F0D0F92A000B212000024B13
:1091000000F0E5FA07B030BDC795001110B50A00B0
:109110001121024B00F0DBFA10BDC0461B96001176
:1091200013B50B0011006A4613706B46040006224B
:10913000581C02F0B1F96A4608212000014B00F0EA
:10914000C6FA13BD3B96001110B50A001121024B5F
:1091500000F0BDFA10BDC0468B9600117FB505002A
:109160000B4BAA00D4580800002C0FD0666F237F49
:10917000E28821780396266F0296E66E0196A46E29
:109180000094FDF709FC2800FFF7FAFD7FBDC046FB
:109190001068FF1F10B51721FFF7E0FF10BD00009A
:1091A00070B50A000D00064B0221040000F08FFA92
:1091B000060029782000FFF7D1FF300070BDC046BF
:1091C0006B95001170B586B000236A4613708368F2
:1091D00004001D78681E0A2859D801A902F04CFB2A
:1091E000060633373B3F43474B4F5300180000F010
:1091F00042F9062312284BD000281BD16088FFF7C4
:10920000D9F90823002813D04279002A47D1264BE8
:109210001A78072312070BD5244B1A680723002A54
:1092200006D01668002E03D0290001AAB04703001B
:109230006A4613706B461B786088002B2AD1FFF7B3
:1092400067FC06B070BD180000F06CF9D4E7180098
:1092500000F087F9D0E7180000F093F9CCE7180088
:1092600000F0ADF9C8E7180000F0C3F9C4E7180032
:1092700000F0F6F9C0E7180000F0F6F9BCE71800B6
:1092800000F013FAB8E7180000F013FAB4E7072368
:109290006A46137069466088FFF782FFD1E70523AD
:1092A000012AC5D1024BB8E79D66FF1F0868FF1F62
:1092B0000C68FF1FF8B52C4F8600F35904000D0011
:1092C000002B40D0DA8882423DD15A78062A33D129
:1092D0001A78002A2ED0012099681A6A097D014265
:1092E00006D0157B054203D007225A700120F8BD35
:1092F0000220014204D0157B054201D00922F4E787
:109300000420014204D0127B024201D00B22ECE780
:10931000164B1B68002BE9D05B68002BE6D02000C1
:109320009847BB5900215B78122BDFD12000FFF753
:1093300015FFDBE70E4BECE7112A04D1002900D022
:1093400032252900F2E7002D08D12000FFF732F97D
:10935000002803D010230279134303712100280051
:10936000FDF798FAC2E7C0461068FF1F0868FF1FA4
:109370000C68FF1F70B50E4E8500AB590400002B22
:1093800013D01B78002B11D10A4B1B68002B04D083
:109390005B68002B01D02000984773595B78122B33
:1093A00003D100212000FFF7D9FE70BD024BECE78E
:1093B0001068FF1F0C68FF1F0868FF1F094B800023
:1093C000C3581020002B0CD01A6A002A09D09B68C1
:1093D000002B06D0127A1B7E101C9A4200D9181C52
:1093E000C0B270471068FF1F70B503000D00140075
:1093F0000220002A30D000292ED013700B78081DCF
:1094000053704B789370FFF7A7FCE07001200221A6
:109410002B7A23716B7B034063716A7B0A40134391
:10942000042263716E7B1640334363716E7BF608D2
:10943000F600334363712B7B0340A371287B01400B
:1094400000200B43A371297B0A401343A3712A7B9D
:10945000D208D2001343A37170BD10B50A000100F9
:109460000120FFF7C1FF10BD10B50A000100022066
:10947000FFF7BAFF10BD70B506000C000220002EE9
:1094800030D000292ED07378201D0B70B3784B702C
:10949000F178FFF76DFC01223579257271794B1057
:1094A0000800134093401040034388101040800090
:1094B000C9080343C9000B436373B1794B1008001B
:1094C0001340934010400343881002409200C908A3
:1094D0001343C9000B4321202373FCF773FE85421D
:1094E00001D2122070BD2220257AFCF76BFE854246
:1094F000F7D823781820042BF4D86378012BF1D8FF
:109500000020EFE7030010B50220002909D0002B4E
:1095100007D00322481C0A7019000D3201F0BCFF6D
:10952000002010BD03000222080010B5002B06D059
:10953000002904D00E32591C01F0AEFF00221000A9
:1095400010BD030010B50220002909D0002B07D060
:109550000422481C0A7019000C3201F09DFF002003
:1095600010BD10B5FFF7DEFF10BD0300022000297B
:1095700006D0002B04D0052200200A701B784B7007
:10958000704703000220002B08D0002906D05B782A
:1095900000200B70013B082B00D9183070470300E6
:1095A00010B50220002909D0002B07D00622481C44
:1095B0000A7019000A3201F06FFF002010BD10B5CB
:1095C000FFF7B0FF10BD02000B00022010B500290C
:1095D0000ED0002A0CD007211970118859701188FB
:1095E000090A997011180822D81C01F055FF0020B3
:1095F00010BD03000A00022010B5002B0CD000297A
:109600000AD099785878090201431180901CD91C1E
:10961000082201F041FF002010BD030010B5022018
:10962000002909D0002B07D00822481C0A70190015
:10963000921801F031FF002010BD02000B00022043
:1096400010B500290BD0002A09D009211970117812
:1096500018185970511C062201F01EFF002010BD81
:1096600010B5FFF75FFF10BD02000B00022010B520
:10967000002A09D0002907D0517819701118062244
:10968000581C01F009FF002010BD030010B5022096
:10969000002909D0002B07D00A22481C0A701900A3
:1096A000063201F0F9FE002010BD10B5FFF73AFFB9
:1096B00010BD02000B00022010B5002A06D00029C0
:1096C00004D018005178FFF753FB002010BDF0B50F
:1096D00085B017001E006A46062305000800918128
:1096E0009380FEF7C0FC1324011E02900CD03800BA
:1096F000B047041E05D1280001A9FEF76FFA041E29
:1097000002D0029801F0E8FD2800FFF701FA2000DE
:1097100005B0F0BDF0B504008BB00191150000213B
:10972000102202A801F0D8FE334EA700B859002835
:109730003CD0C388A34239D10378002B36D142787C
:10974000062A18D102000100553235310C3006AB23
:10975000FFF7A9FA002829D12000FFF72FFE020009
:1097600006A902A801F098FE200002A902F09CF8C8
:1097700001200BB0F0BD816E002917D00B8A112A91
:1097800028D19D420ED101981231093A01F05CFFB7
:10979000012807D1BB5920009D6EFFF70FFE29005D
:1097A0000200DEE732212000FFF7D8FC2000FEF7A0
:1097B00001FF061E1BD0416A002918D00B8AAB425C
:1097C00015D108220198123101F03EFF01280ED177
:1097D000716A0AE09D42E9D108220198123101F034
:1097E00033FF0128E2D1BB59996E8A7EB9E7200088
:1097F00001F00AFEBCE7C0461068FF1FF0B56B4DD4
:1098000087007E5985B0337802900393002B00D0F7
:1098100087E0B368346A01937078062817D1012273
:109820001B7D134202D0217B114218D10222134228
:1098300002D0217B114251D10422134203D0237B59
:10984000134200D08BE0019B5A7DEB5991E0073821
:109850000428F8D802F010F8032E42678300B36E94
:10986000002B03D11C2001F05FFEB066EB599C6E0B
:10987000002C1CD010220021200001F02DFE0298A7
:10988000FFF79CFD01002000FFF72DFA01F0ECFF2F
:109890002082200008211230FFF725FA0298FFF7F6
:1098A0008DFDA076EB592100D888FFF70FFC082228
:1098B000EB591CE0B36E002B05D01A00198AF08812
:1098C0001232FFF70DFC0222019B197DEB59114268
:1098D0003DD0207B10423AD0073208E0F488FCF7F4
:1098E000DBFD01002000FFF711FC0A22EB595A7042
:1098F000029B9C002A595378073B042B11D8D0882F
:10990000FEF758FE00284ED0C3895A08D2182849BD
:10991000029B0298CB542B5941180433254801F07F
:10992000ABFE05B0F0BDFCF79FFD030001208342B4
:1099300001D100200393EB59DE88FCF79BFD0399CE
:1099400002003000FFF7ECFB019AEB59117D042275
:1099500011420CD0217B114209D00B22C7E7F688B7
:10996000FCF73CFD01003000FFF7EEFB6BE7019ACE
:10997000527D01210A4204D0607B084201D00C22B2
:10998000B5E702210A4204D0607B084201D00E22D2
:10999000ADE704210A4204D0627B0A4201D01022C2
:1099A000A5E71222A3E7FA225200B0E71068FF1FD2
:1099B0001468FF1F739D001110B5064B1A7804231D
:1099C000100018401A4200D00348FFF727FA002081
:1099D00010BDC0469D66FF1F2845FF1F70B50400DF
:1099E000FFF7D4FA051E43D12000FFF77FFA234E7C
:1099F000A400A0598268937CDB0708D50321036A81
:109A00001B790B40012B02D1017F0B430377431DD0
:109A1000D97F8B1E022B0DD8022900D00121C088CE
:109A2000FCF790FF042133591A7F59700A431A77C3
:109A3000280070BD01290CD102231022437000219F
:109A40000C3001F049FD305910213530FFF74BF94A
:109A5000EEE70529ECD10223D118437010220C3017
:109A600001F01AFD04233259117F0B431377EAE703
:109A700008251828DCD1053DDAE7C0461068FF1F2D
:109A8000F0B58BB0059143887E4F9E00F4591500C8
:109A90000493002C15D1012902D000200BB0F0BD99
:109AA000101D57781678FFF757F9EB6832000293CC
:109AB0002B7A0499019300903B002000FCF70CFFE7
:109AC000EBE7E388049A934201D00820E6E7237885
:109AD000012B00D1D4E0059B581E092800D9CFE006
:109AE00001F0CAFE05CE0A29CC506C859AB2290035
:109AF0000498FFF773FFD1E72000290010224530BA
:109B000001F0CAFCB9594B78042B02D1013B4B70D0
:109B1000C3E70B000A00253335320C310498FFF7F8
:109B200095F90498FFF702FA0522431E9841BB59A4
:109B3000C0005A70B2E7200029001022553001F011
:109B4000ABFC049B4F4C9D00295904980A0006ABBE
:109B500055320C31FFF77AF929591022453106A800
:109B600001F072FD012808D10498FFF7F7F905907C
:109B7000002804D106222B595A7005988EE7082335
:109B80000593FAE763780C2B7AD1E36E002B03D1AF
:109B90001C2001F0C9FCE066BB59D86E00286FD0CC
:109BA0001022290001F078FCBB590498DC6EFFF705
:109BB00005FC0D22A076BB595A706EE7E06E0028B6
:109BC0005ED063780D2B5BD12B8808220382A91C01
:109BD000123001F061FCBB599A68517D022211429A
:109BE00026D0186A407B104222D00C32E4E763781A
:109BF0000E2B45D1236F002B03D1162001F094FCCE
:109C00002067BB59186F002803D01022290001F0EB
:109C100043FC0F22BB59CFE763780F2B30D1206F65
:109C20000622691C103001F037FCBB599A68517D3F
:109C30000422114203D0196A497B1142D5D1002177
:109C40000498FFF78BFA28E7636F002B0DD0BB5900
:109C5000586F0028F3D01022290001F01DFC0122CA
:109C6000BB5952425B6F1A61E9E7142001F05CFCBA
:109C7000BB5960675B6F002BE9D126E72978DFE7E6
:109C800007200BE71068FF1F10B5064C207001F08D
:109C90001BFD06212078FDF791FF0348FEF778FCB5
:109CA00010BDC0462368FF1F298E001100200BB293
:109CB00070B50D00834216DA264B187801F09CFB34
:109CC000041E0DD00378922B0ED0A02B37D0224B40
:109CD0001878FF283AD0210001F0BEFC002835D1C9
:109CE00080200002684070BD43780E2B0BD03E2BC5
:109CF000EDD18378052B12D0082BE8D181798088AB
:109D0000FFF7D8FA08E0154B82889A42DFD18368C2
:109D10001878591CFEF7C0FE002817D1D7E7104B62
:109D20001B785B0712D50F4B1B68002B0ED09B686E
:109D3000002B0BD0C289811D80889847ECE7FFF784
:109D400041FAA068002801D001F0C6FA200001F015
:109D5000EBFCC5E72368FF1F2145FF1F182000000B
:109D60009D66FF1F0C68FF1F10B50078FFF712FA01
:109D700010BD10B50078FFF7FDFA10BD0C2343436A
:109D8000084A10B59B185A68002A03D0012901D14E
:109D9000904710BD9B68002BFBD00029F9D1984754
:109DA000F7E7C0464068FF1F10B5162813D80123F7
:109DB0008340094A946B1C439463506B98435063EF
:109DC000D46B20009843012901D120001843D063AF
:109DD000116B0B43136310BD00800040F0B50024ED
:109DE0000127154B85B0DA6B144E03921A6C019261
:109DF000DA64019BE3403B4217D0039DE5403D40C0
:109E00000295E5B202992800FFF7B8FF316A736A3C
:109E1000002908D03900002B01D002997940280090
:109E2000FFF7C2FF01E0002BF9D101340C36172CEB
:109E3000DFD105B0F0BDC046008000402468FF1FA0
:109E400010B5012402002000162A08D8054B5968D5
:109E5000D140214204D01868D0400123184010BDE1
:109E6000186DF9E700800040162807D80122064B3C
:109E70008240002903D0D9680A43DA607047D96864
:109E80009143D960FAE7C0460038004030B5162843
:109E900018D8032444430F4BE25C1B199C785D786F
:109EA00001232D1B0135AB40013BA340A140DB4307
:109EB0000C00122807D8084992005218116819405E
:109EC0002143116030BD054A11680B4023431360E4
:109ED000F8E7C0462FBC001108F0004014F0004025
:109EE000C21F70B5D4B20623092C0BD80125084C2B
:109EF0009540002908D00021FFF7C8FF23682B43B5
:109F000023600023180070BD2368AB43F8E7C04608
:109F100000380040F0B5162826D8214B1B185B7876
:109F2000022B21D1032444431E4A1F4EA35C121965
:109F30009478012215008540B76B013CE4B23D43A3
:109F4000A240B563194C122815D89B0000290CD1EA
:109F500017495B1899680A439A600123205C154AE7
:109F6000834011680B431360F0BD11495B18996879
:109F700091439960F1E70E4B00290DD159690A43CD
:109F80005A61225C1328E8D00123203A93400A4901
:109F9000086803430B60E7E7596991435961F0E7AB
:109FA0002468FF1F2FBC00110080004074BC00110A
:109FB00000F00040A0F00040A4F00040F8B50024FC
:109FC0001B4E1C4D1C4B1B5D012B1FD1184A926967
:109FD000E2401A420BD00122AA5693402200143AC2
:109FE000D2B2022A09D815494A6913434B61013498
:109FF0000C360235172CE5D1F8BD0022AA560F49C0
:10A000009200521891680B439360F0E7022BEED157
:10A01000E7B23800FFF714FF01235840C1B23800FF
:10A02000FFF778FF3800FFF70BFF7077DFE7C046D8
:10A030002468FF1F01BC00112568FF1F00F00040CD
:10A04000012202388240054B002903D059690A4396
:10A050005A617047596991435961FAE700380040E5
:10A0600070B504000D000520162C1AD80021200020
:10A07000FFF7FAFEA31E012B03D801212000FFF7F2
:10A08000DFFF00212000FFF72BFF01220A49A24039
:10A090000A4B4868012D05D102431B194A605D70C7
:10A0A000002070BD9043486002211C1961709969BD
:10A0B00091439961F4E7C046008000402468FF1F87
:10A0C00010B516280AD80122074B8240002906D075
:10A0D00019680A431A600121FFF7C2FF10BD196811
:10A0E00091431960F7E7C0460080004070B5050055
:10A0F0000520162D17D80C2300246B430A4A210093
:10A100009B181C70094B28005B195C70FFF7A8FFB7
:10A110000123AB40200006490A681A430A6005493A
:10A120000A689A430A6070BD4068FF1F2468FF1FD9
:10A13000348000403080004070B504000E00FF28DD
:10A1400013D003250540FFF7D1FF084AA3089B0061
:10A150009B183F22ED00AA40AE40196820009143B1
:10A16000314319600121FFF77FFE70BD18380040B0
:10A17000F8B505000520162D25D80C246C43124B8C
:10A18000E4186368002B03D1A3680D30002B1AD0AC
:10A19000022201270D4B00215B195A7028002770FD
:10A1A000FFF75EFF63681E1E08D0A3683E00002B09
:10A1B00004D02800FFF744FE4640F6B228003100E4
:10A1C000FFF7F2FD0020F8BD4068FF1F2468FF1F65
:10A1D000F7B5C420FF222B4B80001958002491436F
:10A1E0007F3A0A431A508022274F5202274E1A60A4
:10A1F000274B1D5D002D21D0A31E012B03D801216B
:10A20000E0B2FFF71DFF012D18D11F4B9B69E34002
:10A210002B4213D0E3B218000193FFF711FE0100A7
:10A220000198FFF74DFFE3B2143B022B1DD801212B
:10A230007156184A8D405369AB4353613B7F002BE5
:10A240000DD0E5B22800FFF793FF2800FFF7F8FDD7
:10A250007B7F0100834202D02800FFF78FFD01348D
:10A260000C370236172CC3D1F7BD012100237156DC
:10A27000F3568D40074A9B009B189A68AA439A6040
:10A28000DCE7C04600E100E02468FF1F01BC0011CC
:10A290002568FF1F00F0004010B504000520162CB3
:10A2A0000CD801212000FFF7DBFE0123044A002027
:10A2B00011194B70A34091690B43936110BDC046C7
:10A2C0002468FF1F70B50E0015000400FFF70EFF95
:10A2D0000C236343094A20009B189D605E60FFF7D2
:10A2E00047FFF021064B074A8900051E5A5002D04D
:10A2F0002000FFF7FBFE280070BDC0464068FF1F2E
:10A300000000FF1FDD9D001170B5134D07202C7854
:10A31000002C1FD1982221005200280001F0DCFA05
:10A320000123C420FF222B700C4B80001C635C6354
:10A330000B4B1C605C600B4B195891437F3A0A43EE
:10A340001A50802252021A600D20074A074901F074
:10A350006BFA200070BDC0462468FF1F00800040DB
:10A36000A0F0004000E100E0D1A10011BD9F00116C
:10A37000030010B50620072B09D8054A137001F019
:10A38000E3F8D7210020034B034A89005A5010BD3F
:10A390005045FF1F0000FF1F151BFF1F70B51D005C
:10A3A00002240C2910D8094ACA40D2070CD5FBF761
:10A3B00015FF041E08D1059A04992800FBF72AFF0F
:10A3C000FCF798FDFFF7F8FA200070BD12100000AE
:10A3D00030B50D7802232C009C43184201D02B434A
:10A3E0001C0008252300AB43284201D02B00234347
:10A3F00020241D00A543204201D01C4325002A2310
:10A400000D70184204D011781E3B0B43137030BD01
:10A410000028FCD10C2113788B43F7E7F8B51D0019
:10A4200006AB1B88140007AA0E000B201778002B20
:10A4300027D10A78022A49D14A6850781178000257
:10A44000244A08438018042840D801F015FA031262
:10A450001D1B2300F06801F07FF8021CC0B2B84257
:10A4600000D93A1CD2B22000F1682A8001F014F819
:10A4700006E00222F3681B882A8023701B0A63709F
:10A480000020F8BD0622EEE701232B80F3681B783D
:10A490002370F5E7F368002B16D008222A801A886B
:10A4A00022701A88120A62705A88A2705A88120A98
:10A4B000E2709A8822719A88120A6271DA88A2710F
:10A4C000DB881B0AE371DBE72B80D9E701202B80B7
:10A4D000D7E7C04600D6FFFFF7B516000A781D0083
:10A4E00008AB1F880C000123022A18D14A68507853
:10A4F000117800022B4A0843801803280FD801F076
:10A50000BBF902254439E06801F026F8C0B2072300
:10A51000B84204D37B190193152B02DD0D231800DB
:10A52000FEBDE0682A003100C01900F0B5FF6B469F
:10A5300000209B88E268D0541B4B1B68834203D0E9
:10A540001B68834200D098470023E8E70B23002FC5
:10A55000E5D1022DE2D1737832781B021343E26811
:10A560001380114B1B68002BEED01B68002BEBD027
:10A570000120E8E70B23002FD1D1062DCED12A00F0
:10A580003100E06800F088FFDEE70B23002FC6D122
:10A59000012DC3D132787533012AC0D8E3681A700F
:10A5A000D2E7C04600D6FFFF306AFF1F70B50C002F
:10A5B0001500072837D801F05FF9041436361B362A
:10A5C000242E182015290BD8184E162200213000F1
:10A5D00000F082FF22002900300000F05DFF002023
:10A5E00070BD18200229FBD11288114B1A80F6E7A2
:10A5F00018200829F4D10A000E48290000F0CCFEEA
:10A60000EDE718200129EBD10B4B10780B49DA69E3
:10A61000FFF7DEFEE3E718200129E1D1064B1078B1
:10A620000749DA6BF4E70220DAE7C046186AFF1F31
:10A63000CE45FF1FC445FF1F5445FF1F7C45FF1F2C
:10A640009C45FF1F030010B50020DB0704D5072140
:10A65000024A034800F08CF810BDC0468CBC0011C3
:10A660005445FF1F054A03001068002803D0828864
:10A670009A4201D1806870470068F6E7346CFF1F8A
:10A680000A88030008009A4204D08A8804309A425B
:10A6900000D0002070470000F8B5F82200230D4FCD
:10A6A0000D4E7968050042433370994200D07B60BB
:10A6B0000A4C0021200000F00FFF00231A007C60EC
:10A6C000AB4202D100203370F8BD01332280DBB2EF
:10A6D000F834F5E7346DFF1F306DFF1F386CFF1F36
:10A6E00073B56B4601900600684615001980FCF7AB
:10A6F00033FF041E11D1002D0FD07689002E11D00A
:10A700000C2000F011FF00280ED0084A04601368E6
:10A7100086808560002B02D11060200076BD1A0073
:10A720001B68F7E70224F8E71324F6E7346CFF1FF1
:10A73000012100220A4B10B549420A4C1980998028
:10A740009A719A70084B2070012019805A60FFF7A7
:10A75000A3FF2078FCF75EFF0448FDF719FF10BD4A
:10A76000386AFF1F3C6DFF1F346DFF1F1DA80011CD
:10A77000022310B5002802D0FFF7B2FF0300180033
:10A7800010BD0000030010B50020DB0704D5042134
:10A79000024A0348FFF7A4FF10BDC046A0BC001149
:10A7A000D445FF1FF0B50E2687B003930CAB1F886E
:10A7B00002ABF6180500080031000292FDF74EF8D2
:10A7C00004000120002C0FD03088FFF74BFF03005E
:10A7D0000E20002B08D05E68002E05D02100280036
:10A7E000039B029A0097B04707B0F0BD0A4B10B523
:10A7F000984207D10122002352420A808B708A803E
:10A800008B7110BDFFF73CFF0028FAD001235B429B
:10A81000038000238370F4E7FFFF0000F8B5050014
:10A8200001290AD1134E00243388F827AB4219D0EE
:10A8300028001149FFF7DAFF06E0022904D10139A7
:10A84000FDF724FF0028EDD0F8BD3B00634372689C
:10A85000D018D35A002B09D03A00002100F03CFE5A
:10A860000134E4B2054B1B78A342EED801235B42CE
:10A870003380DDE7346DFF1F386AFF1F306DFF1F27
:10A8800010B5FFF7FDFE03000020834200D098784A
:10A8900010BD0000F0B589B01C000EAB80CB03905A
:10A8A0001E8810AB1B78049202930B7A0D00DB0616
:10A8B00016D42B780593022B24D00498FFF7D2FEF0
:10A8C000002812D003689C46002B0ED0029B220069
:10A8D000019329003B00644603980096A04705E0D9
:10A8E0000498FFF7BFFE002802D10E2009B0F0BD8A
:10A8F0008368002BF9D00A22290003989847002882
:10A90000D7D0F3E76B6858781A786B4B0002104386
:10A910009842D2D8043B984210D2684B984242D019
:10A9200015D8674BC0180128C7D80B20002EDDD1E1
:10A93000EB681A7859683A80200028E0614BC0180B
:10A94000032800D979E000F097FF846A789E5E4B77
:10A950009842B2D10B20002EC8D101233B80EB6876
:10A9600031001B7823706889013080B2FCF776FFD4
:10A970003A88031E0ED0017802328A183A80428942
:10A9800062704289120AA27059680278E01C00F0D5
:10A9900083FD06E004323A8031000422601C00F09E
:10A9A0009BFD0020A2E70B20002E9FD1EB6807A99A
:10A9B0001E8804233B80330A300026706370FCF746
:10A9C0004DFF051E28D004AB9A890E2304A95B18FD
:10A9D0003E49C668FCF7B6FF00280BD12B783C48EF
:10A9E0006A680599FBF76CFB002803D1012304AAD0
:10A9F0005B42D3813278022A06D17168201D00F0B3
:10AA00004BFD3B8802333B800E2304AA9B181B8816
:10AA1000A3701B0AE370C4E704ABDE81F4E70B20EC
:10AA2000002E00D062E7E9680398FFF729FF0223B0
:10AA30003B802070000A6070B3E70B20002E00D02E
:10AA400054E70222EB681B883A8023701B0A63706C
:10AA5000A7E7E86800F080FDC2B203000720B24219
:10AA600000D243E70DD00299DBB27118994202DBA4
:10AA7000921BD3B20293029BE9681A003B808919AA
:10AA80005AE70023F6E70B20002E00D02EE707221E
:10AA9000EB683A801A7822705A7862705A88A270ED
:10AAA0005A88120AE2701A792271DA886271DB8898
:10AAB0001B0AA37175E7C0460429000002280000A4
:10AAC00000D8FFFFFFD6FFFF03280000FFFF0000B4
:10AAD000D0BB0011F0B58DB06B460020089120224C
:10AAE0009B5E83423DDAA64B187800F085FC071E7A
:10AAF00032D00378B02B2CD10079023816281FD819
:10AB000000F002FD17001E001E001E0031001E0096
:10AB100096001E001D011E0052011E0073011E0042
:10AB2000CD011E0050021E001E001E008E021E00DF
:10AB3000E302944B94491B8878880B80FBF700F85C
:10AB40003800FCF781FF914B1B68002B01D03800C7
:10AB50009847380000F0E8FD8020089B0002434041
:10AB600018000DB0F0BDF6220021874800F0B4FCBB
:10AB70000BAA3B7B7989388900923A000D32FCF7A9
:10AB800085FD0400804B1B78002C3FD146E0804BB4
:10AB9000788805937F4B4100CB5A0BAE073BDBB265
:10ABA00032880293002301937B4B2100069300938C
:10ABB000059BFFF76FFE744D002810D1069B3A8A63
:10ABC0001B889A420BD138000599123000F03CFDE9
:10ABD000002804D02B7862899B00EB185A8016233A
:10ABE00006A81B18328820007989FCF7ABFE2B7869
:10ABF00004009A00AA1851880029C3D00133DBB29F
:10AC00002B70002807D006A9C98A9180634A128850
:10AC10009A42BCD802E0012149429180002B04D025
:10AC200059497888FAF7C0FF8AE73E890A2479E013
:10AC300000253E89574B06937B88069A5B009B5AFA
:10AC4000033B9D4202DB002DF0D05BE0162206A8FC
:10AC500012183B7B798900923A0030000D32FCF7E4
:10AC600015FD0590002858D04689017A7888FCF7B0
:10AC7000D7FC041E44D1464B78880793069B4100BD
:10AC8000C95A454B0439C9B206AAD28A0693029121
:10AC9000019400930599079BFFF7FCFD041E2FD13B
:10ACA000069B39491A88931C002D26D14B80798840
:10ACB000384B4900CB5A5119033B8B4220DD059B91
:10ACC00031485B8941190B71A91C0135C9B2EDB23C
:10ACD000059145191B0A2B71059B2D490433181842
:10ACE00000F0DAFB2C4B059A1B88D318DDB22C4BF5
:10ACF0009E4205D00136B6B29CE749889942D6D02B
:10AD0000002D0CD0204C2800618800F06DFB2070D5
:10AD100021007888FAF758FF12E7059CF0E7002C2D
:10AD200000D183E77B78142B00D109E716493B79E2
:10AD30004E800B700C717888FAF7F8FE00E7162445
:10AD400006ABE41821003889FCF788FD011E00D10C
:10AD5000B7E1788822880F4C45002C5B0A4D013CF6
:10AD6000E4B2029400240F4B01940095FFF792FD8A
:10AD7000041E00D014E129007888FAF735FFDFE6D9
:10AD80003C6DFF1FC044FF1F406AFF1F346AFF1F56
:10AD90003A6BFF1F7066FF1F306CFF1FBE44FF1F22
:10ADA000FFFF0000426AFF1F162406ABE4182100D3
:10ADB0003889FCF753FD011E00D182E17888228892
:10ADC000AE4C45002C5BAE4D013CE4B202947C8954
:10ADD000AC4B01940095FFF75DFD041E00D0DFE051
:10ADE00029007888FAF70AFFAAE60025A44B1D80FF
:10ADF0003B00FE331B78A24A78880792AB4208D901
:10AE00009E4B12880693069943005B5A013B9A4277
:10AE100003DB0799FAF7FCFE92E616246B00FB1899
:10AE2000059306ABE418059B21001889FCF716FD75
:10AE3000011E03D1059B01241E8973E77888924B7C
:10AE40002288069C099343001B5B904E013BDBB2BA
:10AE50000293002300960193099BFFF71BFD041E3C
:10AE600002D0059B1E895DE77B88069A5B009B5A92
:10AE7000079A108832881218934202DC1B1A013B91
:10AE800033807F4C023032880999001900F004FBAE
:10AE90002388328801359B182380EDB2A8E70BAADE
:10AEA0003B7B7989388900923A000D32FCF7EEFB42
:10AEB00000250590059B002B04D10A24002D00D10C
:10AEC0006EE060E0059B7888197AFCF7A9FB010029
:10AED000041E63D1694C6C4B788806940993069BD9
:10AEE0004400E45A694B063CE4B20BAE3288079347
:10AEF0000294019100930599099BFFF7CBFC041E76
:10AF00004CD1079B5E491B881A1D002D30D14A8009
:10AF1000059B5B4C5A8963191A716B1C9BB2E31831
:10AF2000120A1A71162306A832881B187989059807
:10AF3000FCF708FDFF21AA1C2E1D03350B00059010
:10AF400092B2B6B2ADB2002803D006ABDB8AD9B25A
:10AF50001B0AA218651911712B714C4D301D2A88DE
:10AF60004949201800F098FA2B88F618B5B2A1E7E5
:10AF70004988914207D17A8806995200525AEB18B3
:10AF8000053A9A42C4DC3E4C2800618800F05CFA25
:10AF9000207021007888FAF745FED1E5002DF2D126
:10AFA0003E89BFE6162606ABF61831003889FCF755
:10AFB00055FC3D000400FF3500282DD0037A9B0688
:10AFC0000CD400227B893989788800923A000C32AF
:10AFD000FFF7E8FB041E10D03E8915E03088FFF72C
:10AFE00041FB00281AD08368002B17D021001222C1
:10AFF00078889847041EE4D0EEE7AB78002B02D1A6
:10B000007888FAF71FFE0026AB78002B00D097E572
:10B01000002C00D194E585E60124DDE70E24DBE772
:10B02000162506ABED1829003889FCF717FC041E1D
:10B0300047D0037A9B0611D4154A7B881188994220
:10B0400003D01448814207D11380134BF8261D7892
:10B050000023D9B2A94221D30924A1E72888FFF708
:10B0600001FB00282FD08368002B2CD02100122256
:10B0700078889847041EDFD092E7C0467066FF1FAD
:10B08000406AFF1F426AFF1F3A6BFF1F306CFF1FB1
:10B09000346DFF1FFFFF0000306DFF1F310059436B
:10B0A000546801336018615A0029D2D13C00083439
:10B0B0002100F82200F0F0F921007888FAF7CAFDA3
:10B0C0003EE501246CE70E246AE71D4B1A887B8855
:10B0D0009A4231D07888FAF7C7FD31E5F823059810
:10B0E00051684343CD18C95A00291FD03B7A012B20
:10B0F0000BD16C88AB887888AA1D0094FFF752FBAF
:10B10000041E02D000233B722E88F8220021280062
:10B1100000F0E2F900232B80059B0133DBB205939D
:10B12000084B05991B78064A8B42D7D801235B420E
:10B130001380002CCED0F5E5002634000596EFE70D
:10B14000346DFF1F306DFF1F70B504000E00150039
:10B15000FFF796FA031E08D131000548FFF790FA71
:10B1600003001120002B02D01C8000209D7070BDB8
:10B17000FFFF0000F8B50B4F06003B780D001400F0
:10B18000FF2B0ED00A2000F0A7FA011E09D0B12330
:10B190000380002346800371C5800481387800F065
:10B1A0005BFAF8BD1546FF1FF7B50F0008A90600AA
:10B1B000088809A90B240988002821D10234022B10
:10B1C0001ED1557813782D021D432B008B4301931C
:10B1D0007334002B14D1FB68300019000093FFF783
:10B1E0004FFB019C85420BD02A0030000099FFF7ED
:10B1F000ABFF041E04D12A0030007989FFF7BAFFA3
:10B200002000FEBDF0B50E7885B003900AA8058831
:10B210000120022E0DD14C682778647824023C432B
:10B22000054FBC4205D10398DBB201960095FFF7AC
:10B23000BBFF05B0F0BDC0460229000010B50400F8
:10B240000C4800F089FA0C48A16B00F085FA0B4815
:10B25000E16B00F081FA0A48216C00F07DFA094B9D
:10B260000948196800F078FA084B1B68002B00D0D9
:10B270009847FEE7A2BA0011B8BA0011C7BA001188
:10B28000D6BA001104ED00E0E5BA0011406DFF1FD1
:10B29000002307B501A80193FFF7D0FF044A054832
:10B2A000002110B5121A00F017F9F8F783FBFEE73A
:10B2B000446DFF1F1846FF1F01B40248844601BCBD
:10B2C000604700BF3939FF1F01B40248844601BC02
:10B2D000604700BF4D1F000001B40248844601BC16
:10B2E000604700BFD949010001B40248844601BC4F
:10B2F000604700BFA54F010001B40248844601BC6D
:10B30000604700BF291C000001B40248844601BC0C
:10B31000604700BF8B52010001B40248844601BC63
:10B32000604700BFEDA5000001B40248844601BC9F
:10B33000604700BFC56D010001B40248844601BCEE
:10B34000604700BF017F000001B40248844601BC91
:10B35000604700BF156B010001B40248844601BC80
:10B36000604700BF056A000001B40248844601BC82
:10B37000604700BFD13CFF1F01B40248844601BCB6
:10B38000604700BF456B010001B40248844601BC20
:10B39000604700BF8552010001B40248844601BCE9
:10B3A000604700BF810E000001B40248844601BC22
:10B3B000604700BFB54C010001B40248844601BC9F
:10B3C000604700BF691F000001B40248844601BC09
:10B3D000604700BFDD30FF1F01B40248844601BC56
:10B3E000604700BF5118FF1F01B40248844601BCEA
:10B3F000604700BF350E000001B40248844601BC1E
:10B40000604700BFF54E010001B40248844601BC0C
:10B41000604700BF091B000001B40248844601BC1C
:10B42000604700BFDD66010001B40248844601BCEC
:10B43000604700BF7918000001B40248844601BC8F
:10B44000604700BF9DA9000001B40248844601BCCA
:10B45000604700BF090E000001B40248844601BCE9
:10B46000604700BF8D12000001B40248844601BC51
:10B47000604700BF2146010001B40248844601BC78
:10B48000604700BF5952010001B40248844601BC24
:10B49000604700BF014C010001B40248844601BC72
:10B4A000604700BFE94C010001B40248844601BC7A
:10B4B000604700BF6571010001B40248844601BCC9
:10B4C000604700BFD1A5000001B40248844601BC1A
:10B4D000604700BF9130FF1F01B40248844601BCA1
:10B4E000604700BF154D010001B40248844601BC0D
:10B4F000604700BF6932FF1F01B40248844601BCA7
:10B50000604700BF5125000001B40248844601BCD9
:10B51000604700BFF93CFF1F01B40248844601BCEC
:10B52000604700BF3555000001B40248844601BCA5
:10B53000604700BF3D4B010001B40248844601BC96
:10B54000604700BFB352010001B40248844601BC09
:10B55000604700BF151BFF1F01B40248844601BCB1
:10B56000604700BFDD52010001B40248844601BCBF
:10B57000604700BFE134FF1F01B40248844601BCAC
:10B58000604700BF413AFF1F01B40248844601BC36
:10B59000604700BFC53F000001B40248844601BCBB
:10B5A000604700BFC94A010001B40248844601BC9B
:10B5B000604700BFB14E000001B40248844601BCA0
:10B5C000604700BFC51D000001B40248844601BCAD
:10B5D000604700BF813AFF1F01B40248844601BCA6
:10B5E000604700BF0D52010001B40248844601BC0F
:10B5F000604700BFED4A010001B40248844601BC27
:10B60000604700BF5522000001B40248844601BCD7
:10B61000604700BFA93BFF1F01B40248844601BC3C
:10B62000604700BFD91B000001B40248844601BC3A
:10B63000604700BF4135FF1F01B40248844601BC8A
:10B64000604700BF8538FF1F01B40248844601BC33
:10B65000604700BFCD4C010001B40248844601BCE4
:10B66000604700BF594F010001B40248844601BC45
:10B67000604700BFB537FF1F01B40248844601BCD4
:10B68000604700BFA946010001B40248844601BCDE
:10B69000604700BF6DBC000001B40248844601BC95
:10B6A000604700BFE928000001B40248844601BC9D
:10B6B000604700BF3D18000001B40248844601BC49
:10B6C000604700BF2526000001B40248844601BC43
:10B6D000604700BFC926000001B40248844601BC8F
:10B6E000604700BF1D4D010001B40248844601BC03
:10B6F000604700BF9137FF1F01B40248844601BC78
:10B70000604700BFF94C010001B40248844601BC07
:10B71000604700BFD53BFF1F01B40248844601BC0F
:10B72000604700BF75A9000001B40248844601BC0F
:10B73000604700BF434D010001B40248844601BC8C
:10B74000604700BF093AFF1F01B40248844601BCAC
:10B75000604700BF1147010001B40248844601BCA4
:10B76000604700BFE53A010001B40248844601BCCD
:10B77000604700BFC521000001B40248844601BCF7
:10B78000604700BF4550000001B40248844601BC38
:10B79000604700BFC9A9000001B40248844601BC4B
:10B7A000604700BFF539FF1F01B40248844601BC61
:10B7B000604700BF5147010001B40248844601BC04
:10B7C000604700BF3136FF1F01B40248844601BC08
:10B7D000604700BF8132FF1F01B40248844601BCAC
:10B7E000604700BF4551010001B40248844601BCD6
:10B7F000604700BFC95C010001B40248844601BC37
:10B80000604700BF851F000001B40248844601BCA8
:10B81000604700BF2124000001B40248844601BCF7
:10B82000604700BFA134FF1F01B40248844601BC39
:10B83000604700BF0933FF1F01B40248844601BCC2
:10B84000604700BF5549010001B40248844601BC6D
:10B85000604700BF7D18FF1F01B40248844601BC49
:10B86000604700BF055E000001B40248844601BC89
:10B87000604700BF2951010001B40248844601BC61
:10B88000604700BFE53CFF1F01B40248844601BC8D
:10B89000604700BF5D17000001B40248844601BC48
:10B8A000604700BFE548000001B40248844601BC7F
:10B8B000604700BF311B000001B40248844601BC50
:10B8C000604700BF2D3BFF1F01B40248844601BC06
:10B8D000604700BFC132FF1F01B40248844601BC6B
:10B8E000604700BFB70E000001B40248844601BCA7
:10B8F000604700BF1D4B010001B40248844601BCF3
:10B90000604700BFADAE000001B40248844601BCF0
:10B91000604700BF0124000001B40248844601BC16
:10B92000604700BFE117000001B40248844601BC33
:10B93000604700BFC13AFF1F01B40248844601BC02
:10B94000604700BFF30E000001B40248844601BC0A
:10B95000604700BF0189000001B40248844601BC71
:08B96000604700BF090E000062
:10B96800000201030203030304030502060207029F
:10B97800080209000A030B030C020D020E030F0351
:10B98800100311031303140315001600993D001149
:10B99800CD3D00110000000002000000AAB900110E
:10B9A800192A0F180A000000F1590000FD240000B0
:10B9B80041460100997C0011AD9C001101710011F4
:10B9C8009D7A0011A9520011D5AA0011414F00110A
:10B9D800E13F00111141001100000000161600009F
:10B9E80002000000F4B90011F4FFF3FFD2FC0000DC
:10B9F800DD4100110000000000000000547579616D
:10BA08000042312E3000303030310067697468757B
:10BA1800622E636F6D2F707676780042544830310D
:10BA2800000000000200000040BA0011292A282A5C
:10BA3800272A262A252A242A0A180000E2040000B8
:10BA48007102000078EC000074400000102700002C
:10BA580060F0000006640000204E000000000000B6
:10BA6800010000001F501D00023CB400000114003A
:10BA7800100000008102000030313233343536378F
:10BA88003839414243444546005048592B363258CC
:10BA980058504C555330353034005B48617264203F
:10BAA8006661756C742068616E646C65725D0A000D
:10BAB8004C522020203D203078253038780A00501C
:10BAC800432020203D203078253038780A00505314
:10BAD8005220203D203078253038780A00494353D9
:10BAE80052203D203078253038780A00AD560011B4
:10BAF8000157001100000000020000000CBB0011FB
:10BB08006F2A6E2A1A18000001A000000000000029
:10BB18006410B71DC8206E3BAC30D9269041DC7646
:10BB2800F4516B6B5861B24D3C7105502083B8EDF0
:10BB380044930FF0E8A3D6D68CB361CBB0C2649B14
:10BB4800D4D2D38678E20AA01CF2BDBDFB349B5F39
:10BB5800800000800010000000000000035D00115C
:10BB68008D730011275D001195770011AB5D0011F1
:10BB78006B770011215E001141770011735E00118F
:10BB880009790011DB5E0011097900110D5F0011C0
:10BB9800C3780011215E0011F9760011995E001139
:10BBA800A178001100000000000000007F5F001174
:10BBB800A1780011E15F0011A5730011052A042A7C
:10BBC800012A002A02290328012800280118001840
:10BBD80000000000000000000000000000000087D6
:10BBE8000101020102010102010203030401030130
:10BBF800010101010303020103000D000E00100002
:10BC0800110013001401070108010A010B011C01AE
:10BC18001D02040205020702080219021A021C0288
:10BC28001D030103020317000201000504000807B1
:10BC3800000B0A001716001D1C0102010105040172
:10BC48000E0D011110011413011716011A19020221
:10BC580001020B0A020E0D0211100214130217162C
:10BC6800030504030807030B0A030E0D0001020372
:10BC780007090A0B0E0F101112141718191A1B1F97
:10BC8800202122001DA40011D9A4001100000000E9
:10BC980002000000D6BB00110000000005B2001130
:0CBCA8000000000002000000D4BB0011EE
:020000041FFFDC
:1000000000000000F53E0011B0B90011ACB90011BC
:100010002463FF1F0000000000000000000000003B
:1000200000000000000000000000000000000000D0
:1000300000000000000000000000000000000000C0
:1000400000000000000000000000000000000000B0
:1000500000000000000000000000000000000000A0
:100060000000000000000000000000000000000090
:100070000000000000000000000000000000000080
:100080000000000000000000000000000000000070
:100090000000000000000000000000000000000060
:1000A0000000000000000000000000000000000050
:1000B0000000000000000000000000000000000040
:1000C0000000000000000000000000000000000030
:1000D0000000000000000000000000000000000020
:1000E0000000000000000000000000000000000010
:1000F0000000000000000000000000000000000000
:1001000000000000000000000000000000000000EF
:1001100000000000000000000000000000000000DF
:1001200000000000000000000000000000000000CF
:1001300000000000000000000000000000000000BF
:1001400000000000000000000000000000000000AF
:10015000000000000000000000000000000000009F
:10016000000000000000000000000000000000008F
:10017000000000000000000000000000000000007F
:10018000000000000000000000000000000000006F
:100190000535FF1F5533FF1FC16601000000000039
:1001A000000000000000000000000000000000004F
:1001B000000000000000000000000000000000003F
:1001C000000000000000000000000000000000002F
:1001D000000000000000000000000000000000001F
:1001E000000000000000000000000000000000000F
:1001F00000000000000000000000000000000000FF
:1002000000000000000000000000000000000000EE
:1002100000000000000000000000000000000000DE
:1002200000000000000000000000000000000000CE
:1002300000000000000000000000000000000000BE
:1002400000000000000000000000000000000000AE
:10025000000000000000000000000000000000009E
:10026000000000000000000000000000000000008E
:10027000000000000000000000000000000000007E
:10028000000000000000000000000000000000006E
:10029000000000000000000000000000000000005E
:1002A000000000000000000000000000000000004E
:1002B000000000000000000000000000000000003E
:1002C000000000000000000000000000000000002E
:1002D000000000000000000000000000000000001E
:1002E000000000000000000000000000000000000E
:1002F00000000000000000000000000000000000FE
:1003000000000000000000000000000000000000ED
:1003100000000000000000000000000000000000DD
:1003200000000000000000000000000000000000CD
:1003300000000000000000000000000000000000BD
:1003400000000000000000000000000000000000AD
:10035000000000000000000000000000000000009D
:10036000000000000000000000000000000000008D
:1003700091B2001100000000000000000000000029
:10038000000000000000000000000000000000006D
:10039000000000000000000000000000000000005D
:1003A000000000000000000000000000951AFF1F80
:1003B000000000000000000000000000000000003D
:1003C000000000000000000000000000000000002D
:1003D000000000000000000000000000000000001D
:1003E000000000000000000000000000000000000D
:1003F00000000000000000000000000000000000FD
:081838005071FF1F4118FF1F52
:10184000024981F3088802F083FB00005071FF1FFA
:1018500010B502F0B5FA072804D0122808D00228E3
:1018600008D010BD044A0420136B01331363F8E75A
:101870000220F6E71420F4E71867FF1FF8B5070009
:101880000C0026002500503630785135002804D150
:101890000300287058342370F8BD2978CA00481E08
:1018A0008141A3183800A25C5B68C9B2FFF7D0FF82
:1018B00000280DD12B78DA00A218013350602B706C
:1018C0003378044A013B3370136A01331362D8E75B
:1018D0000123DFE71867FF1F5C234343074910B567
:1018E000C9180B0058331B78012B05D1FFF7C6FF31
:1018F000034A936A0133936210BDC0464C67FF1FD1
:101900001867FF1F10B502F013FB064A01211300F0
:1019100010CB4942D967044B136002F071FA2000E2
:1019200010BDC04600E100E01000100010B504003A
:1019300002F0FEFA024B1C6002F062FA10BDC046D3
:1019400000E100E010B5040002F0F2FA4021094A7B
:10195000200013688B43136002F012FA01F0B4FD0B
:101960000022054B01201A60044B04321A6002F079
:101970006FFCFEE71CF00040C4F00040C0F00040E7
:10198000431E5A425341A022F0B5D2015B4213409C
:10199000154D164A40019B182A18127E8BB00191F2
:1019A000002A1BD01A000832D46F0022E6B206AF1C
:1019B000E4B294420EDC2818C369002B08D00199C8
:1019C00002AA117106AA049202AA167303A89847E4
:1019D0000BB0F0BD1978B9540132EAE71A7D1A78D4
:1019E00006AB01261A70E6E7D869FF1F00400040E9
:1019F000F0B5254B04004001C25C85B0002A2BD015
:101A00001A18117E002927D0917E002924D011793F
:101A1000022921D11689D788D168F51BADB22A1CBD
:101A2000102D00D9102292B2BE4217D118180123EE
:101A300003710023C269C38003819A4206D06846BD
:101A4000032103730171029301A890470820002C21
:101A500000D0192001F034FC05B0F0BD013C654216
:101A60006C41A0256442ED012C40084D1B186419FF
:101A7000074D0633013A92B2AA42EDD01888461CAF
:101A80001E80085C2070F5E7D869FF1F0040004009
:101A9000FFFF00000F220E4B10B59868104002386F
:101AA0000A280BD802F01EF90D0A0B0A0A110A0ABD
:101AB0000A0A060002210020FFF762FF10BD012183
:101AC000F9E70020FFF794FFF8E7DB6FF6E7C04681
:101AD000004000400F220E4B10B5986810400238AD
:101AE0000A280BD802F0FEF80E0A0B0A0A120A0A9C
:101AF0000A0A060002210120FFF742FF10BD012162
:101B00000800F9E70120FFF773FFF7E7DB6FF5E760
:101B10000090004013B5334C2378072B3DD8324B4F
:101B20001A78324B002A39D18022196852020A43AE
:101B30001A60252001F084FF20232D4A11680B43F1
:101B4000802113606B460422C905086807331042E0
:101B500028D080210422C905C86810422ED08021D7
:101B60002020C905CA688243CA6014221A701A78F4
:101B7000002A2FD18021C905C86820320243CA60DB
:101B800014221A701A78002A28D11A4B1A7D22784A
:101B90005A601D221A705932DA6013BD1A6816494C
:101BA0000A40C5E7086802430A6014221A701A78CE
:101BB000002ACED01A78013AD2B2F7E7C8680243B9
:101BC000CA6014221A7019784A1ED2B21A700029FB
:101BD000F9D1C4E71A78013AD2B2C7E71A78013AC4
:101BE000D2B2CEE75045FF1F1846FF1F3CF0004021
:101BF0004845FF1F00200040FFFFFEFF564B70B519
:101C00001B68012B03D1554A936D0133936502F094
:101C100007FB534B534A1860534B544C1A60012333
:101C2000534A1360534A13602378002B06D00622D0
:101C30005149524802F0D4F900232370504A514BC5
:101C400010681B78C1B2002B0ED14F4CC0B2237864
:101C50005BB2002B4FDB237824785BB264B21B04A9
:101C600024021B191B1813600B1C50294ED950233A
:101C7000464A47491078DBB2FF2202284BD1086858
:101C8000444C454D267890432A78964254D9227880
:101C900024782E78023B5D10A31B6B435201D31AAC
:101CA00010335B111843086002F02AFA031F012B5E
:101CB00045D83A4B1B78002B06D0394B1B78002BAC
:101CC00002D0002002F0CCF8A122364B9200997885
:101CD000354B4A431B689B18832292009B181B7844
:101CE000033B012B03D8AF20400002F009F9012289
:101CF0002E4BDA8270BD237824785BB264B2FF3356
:101D0000FF341B0424021B190138ABE7CAB2022AB4
:101D1000AED20223ACE70868254C264D26789043C6
:101D20002A78964208D9227824782D78023B5B10D5
:101D3000641B63435201B2E72378DBB2B2E70228A7
:101D4000D5D11D4B1B78013B022B03D91B4B1B78B4
:101D5000022BCCD16C20C8E79809FF1FFC0FFF1F96
:101D60005066FF1FFF3F0000141003405466FF1F22
:101D70000C10034000100340D50BFF1F7211FF1F12
:101D8000B40003408C09FF1F680AFF1F490AFF1FA8
:101D900094000340460AFF1F470AFF1FF908FF1F70
:101DA0002209FF1F300DFF1F3409FF1FBC0BFF1F4F
:101DB000440AFF1F450AFF1F1C09FF1F2309FF1FBD
:101DC00010B501F0E5FF0022014B1A8010BDC0469E
:101DD0004C66FF1F10B501F0A3FFA121054A890041
:101DE0009478054A61431268044B5218528C1A8049
:101DF00010BDC046300DFF1F3409FF1F4C66FF1F8A
:101E000010B50D4B0D4A9978A1239B004B431268E6
:101E1000D218531DD97F0A4B1B88994209D2441C02
:101E200007D0C82805D0D2695B1A5A43054B5343E3
:101E3000C01802F0E5F810BD300DFF1F3409FF1F78
:101E40004C66FF1F7102000070B5244D2B68002BFB
:101E500028D002F015F92B68D8402B680400002B1D
:101E600027D002F0C5F92B68D8401D4B1D4A997840
:101E7000A1239B004B431268D118D25C91239B0095
:101E8000002A20D0CA580132CA50174B17491B6884
:101E90000868834214D3D23B181A012A1AD0144B73
:101EA000186070BD02F0ECF8124B196802F070F87F
:101EB000D3E702F09DF90F4B196802F069F8D4E7F7
:101EC0000D495B18E8E7CA500C4B1B68DB68E41847
:101ED000201AE4E7F530FF30E1E7C0461C08FF1F99
:101EE000300DFF1F3409FF1F9C09FF1F5066FF1FA5
:101EF000A009FF1F1808FF1F2DFF3F005866FF1F96
:101F000070B504000D00282916D10300A433C2883F
:101F10001B889B1A0B4A9BB293420DD906006A3666
:101F200005223100653001F083FF002804D1310023
:101F3000200002F0F5F870BD2900200002F058F8EA
:101F4000F9E7C046FE7F0000F8B50400012001F06B
:101F50007FFF01F0B5FF174A1749106009680300B9
:101F60001648174E01601748776805680020AF4291
:101F700001D27068281A144D091928601348C162EB
:101F8000A421446A49032143416211490978002987
:101F900005D010490978022902D10F3B1360F8BD22
:101FA000012901D1083BF9E7032901D1053BF5E7F8
:101FB000033BF3E7E408FF1F28F00040340AFF1F4B
:101FC00028100040180AFF1F1C0AFF1F00F00040E5
:101FD0001C09FF1F4A0AFF1F70B580241025E40565
:101FE000A3682B43A36001F0DBFFA368AB43A360AE
:101FF00070BD0000F7B5160080221C001023D2052A
:102000000191916805000B43936000225A4BD73031
:102010001A6001F0ADFE9D232A002F009B00EB58B3
:10202000CA3201210092FC37002B01D00021009A16
:10203000386802F03DF82900009BCB311A784F4BED
:10204000D3351A604B780A781B0213438A7812043E
:102050001A43CB781B061343494A1BBA13604B79CA
:102060000A791B0213438A7912041A43CB7931008F
:102070001B061343434A1BBA13606B782A781B0272
:102080001343AA7812041A43EB781B0613433E4A03
:102090001BBA1360019A330213433C4A13603C4B52
:1020A00022001B1B9C4603293DDCB3089A00130049
:1020B0005142B21A032A46D1354AE018511A8278A1
:1020C0004078120400020243E05C043302430A60D9
:1020D0000022FF2B4BDDF0222E4B12011A600F2243
:1020E0002D4B1A602D4A1368002BFCD00023224A86
:1020F00027491360091B321D0B191B68043A180A83
:1021000023706070180C1B0EA070E3700434002A5A
:10211000F2DC802210213B68D20501333B609368DA
:102120008B439360F7BD6346D578981893782D0656
:102130001B042B43157804392B43557804322D02A8
:102140002B430360AFE7022A0AD1114AE05C511A1F
:10215000E2185278120202430A6004339BB2B7E7D6
:10216000012AB5D10A4A521AE15C1160F5E7084923
:1021700059180A600433ACE7000004403C000440F6
:102180003800044034000440300004400C00044097
:102190000001044004000440100004401400044006
:1021A000F7B5150080221C001023D205009191681C
:1021B00007000B4393600023654AD730136001F09A
:1021C000D7FD9D233E009B00F9583B00CA363200E4
:1021D000FC33002900D07FE0586801F069FF390026
:1021E00032785C4BCB311A604B780A781B02134370
:1021F0008A78AC4612041A43CB78281D1B06134379
:10220000554A1BBA13604B790A791B0213438A792A
:1022100012041A43CB791B061343504A1BBA1360AE
:102220004B7A0A7A1B0213438A7A12041A43CB7A36
:1022300021001B0613434A4A1BBA1360009A2B0263
:102240001343484A13602200474B1B1B0093009B1B
:10225000CE785B1801938B7836061B0433430E78D7
:10226000043833434E78043136023343019E3360E1
:102270000328ECDC0321A808431C9B0029408000B4
:1022800003292BD13849E5185E18A9786D78E35CED
:1022900009042D022943194331600300083300214A
:1022A000FF2B2DDD314B324919600F21314B196065
:1022B000012327490B60304B19680029FCD0062107
:1022C0001B680B40042B20D080220020D20593688D
:1022D0000A318B439360FEBD01217DE7022908D1BD
:1022E00021495D18E1184978E35C09021943296026
:1022F000D3E70129D3D11C495918E35C0B60CCE723
:102300001948181801600433CAE7002310490B600C
:102310006346002B0CDC3B00FC335A681021013271
:102320005A608022D205936801208B439360D2E7E4
:10233000009B9B181B68190A13705170190C1B0E17
:10234000D37004235B4291709C440432E0E7C046A2
:10235000000004403C0004403800044034000440C5
:10236000300004400C00044000010440040004401C
:10237000080F0000100004401400044070B5061E51
:1023800019D00222614B9B799343012B13D1604BEF
:102390001A78FF2A0FD15A78FF2A0CD19A78FF2A8F
:1023A00009D1DA78FF2A06D11A79FF2A03D15B799D
:1023B000FF2B00D1A7E0574B0C201A78012A08D038
:1023C0000022554D1A702B781A00093A042A01D8B8
:1023D000212070BD5A1F012AFAD94C4CA07B042839
:1023E00000D990E0A279032A00D98CE0821E012A4C
:1023F00003D862881F2A00D885E0002E61D0012E04
:1024000000D080E0A288012AE2D0002B0AD1013856
:10241000032803D801F066FC151D19151F202E7026
:1024200001F056FE2B785A1E032A16D800253B4B86
:102430001D602823237501F0ABFEA8422ED0A58095
:10244000C6E7022320202B70EAE7042322202B700A
:10245000E6E7032321202B70E2E7073B012BB7D8E7
:102460002F4B1B68DB6A9B06B2D52E4B1A78002ACD
:10247000AED1A27B911E012901D9002AA8D1022246
:1024800080211A702823284D89012878237501F0AE
:10249000DFFD80212878890101F03AFE0123A38025
:1024A000224B1B78002B0AD0FA228021204B92006D
:1024B0001B8809025A431C4B187801F0F1FD0020DB
:1024C00087E701F035FD2B78A680073B012B06D965
:1024D00018482E7001F054FE1E2001F0F9FD114B3A
:1024E000114C1A78002A06D0802100222078890118
:1024F0001A7001F0ADFD01F083FC80212078090203
:1025000001F0A6FDDBE7122063E7C046A60BFF1F24
:102510006B09FF1F1A09FF1F1C09FF1F4809FF1F36
:102520005866FF1F2309FF1F1B09FF1F2109FF1FFB
:102530002C09FF1F0010004010B5002901D001F048
:102540003FFD10BDF7B5604B01919978A1239B0029
:102550004B435E4A060014681022E418D6235B0041
:10256000E0583623FF33E35C00279343222B41D10D
:10257000574B0F3A1A600760012501F089FD019B56
:102580001880E8235B00E35C002B01D0B34258DDE8
:102590000023504FFB70AD33FF33E3581A68002A15
:1025A00003D09B88DB439B071DD03823FF33E35CBC
:1025B000002B18D09B235B00E35C002B13D1D1339D
:1025C000FF33E35CB3420EDAA4235B00E15AE01868
:1025D000090A023101F07CFC23000122FE33013E96
:1025E00001351A87FA70E8235B00E35C002B2AD0E0
:1025F000A8B2FEBD03683D00002BBED08188043028
:10260000090A023101F064FCD6235B00E3581F6025
:10261000B2E72300B133BA00FF33985801378188FD
:102620000430090A023101F053FCE8235B00E35C4B
:10263000BB42EEDCE822F61AED1800235200A35448
:10264000A6E70027F1E7200001F0E2FD00281FD0F7
:10265000002E1DDD7319882647190193B60020004E
:1026600001F09EFB5A3080002018406801358188B7
:102670000430090A023101F02BFC200001F018FCA3
:10268000A3590133A351BD4202D0019B9D42E6D123
:10269000114BE35C002BABD095239B00E35C002B3C
:1026A000A6D00E4BE15A0029A2D00D4AA35C994254
:1026B00002D90133A3549BE700231A212000A3541D
:1026C00001F08EFD94E7C046300DFF1F3409FF1F57
:1026D00000140340E010FF1F5A02000072020000C5
:1026E0005E020000F8B51D4B1D4F1A78002A10D16C
:1026F000BA7B002A02D101321A7003E0032AFAD011
:10270000022AF8D001F044FD00220120154B1A7076
:10271000F8BD154B154D1C68154B9E7801232B7089
:102720002878C0B200F0DEFCBB7B002B0BD101F09F
:10273000B7FBA1239B007343E41883239B00E41899
:1027400023782B70E4E7032B02D101F011FCF0E7B2
:102750000020022BDCD101F0B3FCEAE71C09FF1FCB
:10276000A60BFF1F2309FF1F3409FF1F490AFF1F84
:10277000300DFF1FF0B587B00EAD2F780FAD2D785F
:102780000593AC46634614000E4D0CAA12782E78C1
:1027900003930D9B009201932200059B029701F089
:1027A000B7FB2E70012C01D0042C08D180220649E1
:1027B0008B889343054A1278D20113438B8007B06C
:1027C000F0BDC0461C09FF1F6C11FF1F7809FF1FD9
:1027D0000B001B3B70B504003020E02B0DD813001C
:1027E000E025493BFF3B9BB2ED00AB4205D8034BD4
:1027F000200019825A8201F0ABFA70BD8410FF1FCD
:1028000010B501F00DFD054B00205B68052B04D9C8
:10281000034A5268D20200D4980810BD001000404C
:10282000FCE100E070B501F083FB0D4B1B68FC334D
:10283000DC691D6AFFF7E4FF6419844204D2094B86
:1028400001241B68002B07D004220024064B1A70B9
:10285000064A93690133936101F0D2FA200070BDFA
:102860005866FF1F9809FF1F2309FF1FFC0FFF1F5A
:1028700070B50C4D2B68FC335C6A01F059FBFFF717
:10288000BFFF2B680025FC339B6AE318834204D208
:10289000054B1B68AB4200D1051B01F0B1FA2800C3
:1028A00070BDC0465866FF1F9809FF1FD722044B12
:1028B00092009B5810B5002B00D0984710BDC04621
:1028C0000000FF1FF0B587B001F096F9FFF7EEFFAB
:1028D000CA4BCB4C04931B78022B45D1C94B1B68C8
:1028E000186A01F0B5FAC84BC84A1A60C84BC94A01
:1028F0001A60A022C84B52001A60049B187801F09D
:102900004FFCC649C64801F06BFAC649C64801F0FB
:1029100067FA1022C54BFF201A60802252031A600A
:10292000802292031A60802212041A6001F098FA41
:10293000012001F07DFCFA20400001F001FC58204C
:1029400001F0DEFABA4801F033FB012001F090FB00
:10295000072001F075FA2268B64B1A4084235B0009
:102960001343236007B0F0BD01F092FAB24E02901B
:10297000322001F06DFA33681B0629D43C2001F0A7
:1029800067FA0F2001F064FA9C4B1B78012B00D1F1
:102990001EE180223368A94D134200D0A7E02B68C6
:1029A000032013432B6001F053FA01F071FA029BEC
:1029B0000299C31A5A1E814200D81A00A04B1A600D
:1029C000904B19681E2353439E4A9B18CB618AE79C
:1029D00001F05EFA80239C4ADB02116803900B43EE
:1029E00013602268934B994F1A40282313432360A6
:1029F000032001F02DFA03203D6801F029FA3B681D
:102A00000320DB03DB0B009301F022FA3B68ED03AC
:102A1000DB03ED0BDB0B8E4A0193AB18C22B30D8D6
:102A2000009B9B18C22B2CD8019B9B18C22B28D82B
:102A3000009B2A009D4200D21A00009B9D4200D9B3
:102A40001D00019B934200D21300019A954200D9C8
:102A500015005B1B122B14D80C22336814209343EF
:102A6000336033687B4A1340336001F0F1F9082189
:102A70003B682268DB038A432260774ADB0B1360E2
:102A80007FE7032001F0E4F93B68DB03DB0B0593F0
:102A900001F0FEF9039B0399C21A531E814200D82C
:102AA00013006E4A93421BD9FF23356869492D0AEA
:102AB0001D4032686B1C1B060A401B0C134333601D
:102AC0000C23326800209A43083B1343336001F023
:102AD00047FA6348634BA840984206DCFEF732FF92
:102AE000019B009D0093059B95E75F48F6E7002357
:102AF0005E4F554A3B6080231168DB020B43136035
:102B000080222B68032013432B6001F0A1F93B685E
:102B1000052601333B6080232A685B0213432B6048
:102B20002268444B03201A40514B1343236001F0A9
:102B30008FF90821454B1A682368D2038B43236021
:102B4000454B023900931B68D20B4B439A420CD879
:102B50009B1A3B2B0BD8236846490B4023602B68FC
:102B60000B402B60444B1A601FE7D31AF1E7013E7C
:102B7000F6B2002ED4D123683E4A134023602B685E
:102B800013402B603B68042B07D9BFF34F8F3B4B9F
:102B90003B4ADA60BFF34F8FFEE780222B680320A9
:102BA00093432B6001F054F92268224B03201A4012
:102BB00028231343236001F04BF9244B009A1B6830
:102BC000DB03DB0B1360082223689343236097E742
:102BD00007222C4D2B681340012B02D1002001F05D
:102BE000DFFAAB68284A02201340AB6001F030F9ED
:102BF0008023AA685B001343AB60D6E64A0AFF1F36
:102C00005CF000405866FF1F000003400180063D55
:102C1000BC00034034080000A4000340710200001F
:102C200014100040FFFF3F002810004000E100E0CA
:102C30003075000000FEFEFFC4F0004044F000408C
:102C40004066FF1F7206000040F0004064F0004044
:102C500091FCFFFFFF00FFFF4866FF1FE30C000031
:102C6000E88000005F361E0060361E00B444FF1F7F
:102C700028000100FFFFFEFF4466FF1F00ED00E09B
:102C80000400FA053CF00040FFFEFFFF694E336888
:102C900088331B6883F3088801F0D2FA00F014FC33
:102CA000654B664A1B68934207D0002001F058F933
:102CB0000221634A13688B431360FFF703FE614BE5
:102CC000614C1878C0B201F04BF80023A3600233C6
:102CD000A3605E4B0120236001F0BAF80323A360D8
:102CE00001F0D6F8040001F09BFA050001F0D0F8DD
:102CF000574B186001F084FA564B1968621A531E3C
:102D0000A14200D213008022D203934201D39B023E
:102D10009B0A3268D16AC90700D478E04E491C0C7E
:102D200009689BB24C4359432402090A64180327DB
:102D30004A49FC3293680A6849489B1A494A4A4EF4
:102D400012684A499B18414A34609A183B400193E3
:102D5000036892089C46019B0A6063440360042B4D
:102D600003D901323B400A6003600B684049E41814
:102D7000200001F00DF93F4F3D493B68C3183B600F
:102D80002000019301F054F93B4C206808183849A1
:102D90002060884205D9019B01333B6001F048F96E
:102DA000216001F005FA354B1B78002B0ED001F0A5
:102DB00037FA3168324B4A1B1B6812189A4233D2D9
:102DC000591A4919091A2F4801F00AF82E4C237A8A
:102DD000002B0FD001F024FA3168E3684A1B121867
:102DE000934224D9591A4919091A284800F0F8FFC2
:102DF00000232372264B83F3088801F039F8022060
:102E000001F066F9002001F0ABF801F0E1F9DC0116
:102E100099000234641A5900641A09214B43803323
:102E2000CB40A408E41882E7FA218900CBE71949CE
:102E3000DBE7C0465866FF1F0C0AFF1FB64121039F
:102E400010000040490AFF1F14100040C409000090
:102E5000100AFF1F340AFF1F380AFF1F200AFF1F36
:102E6000280AFF1F1C0AFF1F3C66FF1F240AFF1FC2
:102E7000710200006008FF1F2C0AFF1F1C09FF1FC2
:102E8000E408FF1F00100040740BFF1F3C100040BF
:102E900000000020DC050000A022054B92009B589A
:102EA00010B5002B01D0984710BD01F039F8FBE7B1
:102EB0000000FF1FA122054B92009B5810B5002B6C
:102EC00001D0984710BD01F02BF8FBE70000FF1F71
:102ED000A222054B92009B5810B5002B01D09847B9
:102EE00010BD01F01DF8FBE70000FF1FA322054BFA
:102EF00092009B5810B5002B01D0984710BD01F0EF
:102F00000FF8FBE70000FF1FA422054B92009B581F
:102F100010B5002B01D0984710BD01F001F8FBE778
:102F20000000FF1F70B501F07BF9514B18600420C1
:102F300001F0CEF801F04CF80400C30702D401F010
:102F400007F970BD00224B4B1A604B4B18780138C3
:102F500004282CD800F0C6FE03231B1F27002000E6
:102F600001F0E6F80128ECD0444C2378042B71D111
:102F700000F0E6FF002806D000F082FF582000F0A5
:102F8000BFFF02232370032001F0A2F8D9E720003D
:102F900001F0E6F8E6E7200000F0A2FFE2E72000FB
:102FA00000F0B6FEDEE7200000F0EAFFDAE701F00D
:102FB000A7F80500012808D1314B1B78053B012BF0
:102FC00003D82000FFF768FFCEE72C4B1B78022BBD
:102FD00001D0052B20D1022D28D12A4B9B7BAB435E
:102FE0001CD12000FFF766FF254B18780128BBD1C4
:102FF0006405B9D4234925224B7B034205D1233AEA
:1030000013405A42534126331A000B7D9342ABD9E9
:10301000322000F08DFEA7E7022D07D1184B1B7858
:10302000052B11D12000FFF753FFDDE7012D0BD158
:10303000012B03D12000FFF759FF95E7062B03D1A1
:103040002000FFF761FF8FE7200000F069FF022DED
:103050008AD1C9E7032B04D10B4B987C01F0B0F85F
:1030600091E7072B8FD1094B987B00F0A1FE8AE7EF
:103070009C09FF1F9809FF1F9009FF1F2309FF1FCD
:103080001C09FF1FA60BFF1FBC0BFF1FD40BFF1F4C
:10309000FA210A4B0A4A49001A640A4A5A500A4A53
:1030A00004395A50094A08319A64094A5A50094A5F
:1030B0005C315A50084ADA667047C0460000FF1F6C
:1030C0007527FF1F7128FF1F2528FF1F7D23FF1F66
:1030D000E526FF1F011EFF1FD51DFF1F10B500F0C5
:1030E000E9FD10BD8023F7B59C46264B264F019382
:1030F0002649274A274D284C284B02281AD16046DA
:1031000038600868264E3040802636033043086019
:1031100001990978002909D11660224A2A60224AB9
:103120002260E02219689143A03A1BE08021C90285
:103130001160F2E766463E600F68194E3E408027F8
:10314000FF023E430E600199097800290DD11760F6
:1031500001280ED1154A2A60154A2260E02219681A
:103160009143C03A0A431A60F7BD80218902116079
:10317000EEE7E0210F4A02432A600F4A22601A68F4
:103180008A43F0E74B0AFF1FE0000340D8000340EA
:103190009000034000000340500003404000034003
:1031A000FFFFE3FF0280063D804508220180063DC7
:1031B000806608220080069880550822F8B51E4BCC
:1031C00080261A68002014003440324232D11A6836
:1031D0001A4F32431A6001223B68063093433B602A
:1031E00000F036FE0122164D2B681E432E603B6810
:1031F0000A2613433B608027BF00124B1B683B42EB
:1032000011D1013EF6B2FF2E09D17E220E4B1C6871
:103210002B68E40B1440934323432B6005E0082004
:1032200000F016FEE9E7002EEFD180222B6860083F
:1032300093432B60F8BDC046C4F000405CF00040F2
:1032400018F0004068F0004060F0004010B500F059
:10325000E7FE01215820034A00F04AFEFFF7AEFFC7
:1032600010BDC046600AFF1F10B578220021034838
:1032700000F0AEFD00F0E4FE002010BD6069FF1F0D
:1032800070B5040000F054FE00230C200B4A01002E
:1032900059438D18515C00290DD0A14208D101235A
:1032A00000246B7000F0A4FD00F0AAFD200070BDAA
:1032B00001330A2BEBD11224F6E7C0466069FF1FE9
:1032C00070B5040000F034FE002319001D000D4A03
:1032D0001078002806D0A0420CD1557001310C3274
:1032E0000A29F5D1002B0AD100F0AAFE00F088FDD2
:1032F000002070BD5078461EB0411B18EEE700F06C
:1033000077FDF3E76069FF1FF7B504000C20002389
:1033100084460E4D019267465F43E85D7E19A042E8
:1033200012D000280BD10A4B9C4662461B7808330A
:103330001370019B70707C557160B360FEBD0133EA
:103340000A2BE8D10320F9E70720F7E76069FF1FA0
:103350005C69FF1F8021F8B5464BC9051B68C12475
:103360008B60454BFF261A68012313434B61434B87
:10337000A4001A68424B40201A60424B1A68424B24
:103380001A60424B1A59B2431A51C52292009D58F5
:10339000B5432843802598509F583D48ED0107408C
:1033A0003D439D509D5880272D022D0A2943995059
:1033B00080211A59090202400A431A5104341A5949
:1033C000344D3F042A403A4380271A511A593F0688
:1033D0001202120A3A431A5108341A5902400A4397
:1033E0001A51C32292009D58B5432C0080252C43CE
:1033F0009C509D582C0004400C439C509D58254CDB
:1034000025408024240425439D509C588025240277
:10341000240A3C439C50C424A4001A59B2432A43B2
:103420001A511A591202120A17431F5108341A5915
:10343000B24315431D5100251A5902400A431A513F
:1034400004341A59024011431951134C134B1B7881
:10345000DB08AB4201DC0020F8BD2378002B06D04E
:10346000A368002B00D0984701350C34EEE71220FA
:10347000F2E7C0464C45FF1F4845FF1FB0F0004033
:103480005869FF1FB4F000405469FF1F00E100E0DD
:10349000FF00FFFFFFFF00FF6069FF1F5C69FF1F68
:1034A000030010B51F2809D8072200201340072465
:1034B00004490A78A24313430B7010BD0023062071
:1034C000F5E7C0465C69FF1F034A04491368002002
:1034D0000B4013607047C0461CF00040FFFFC1FF67
:1034E000054B06491B780A6805485B0702401B0B21
:1034F000134300200B6070475C69FF1F1CF0004005
:10350000FFFFC1FF70B50C25FFF7EAFF0A4B1C78DF
:103510000A4BE4086543ED18002C01D1200070BD72
:103520002B78002B06D06B68002B00D09847013C0D
:103530000C3DF1E71220F2E75C69FF1F5469FF1FA1
:1035400007B50422074801A900F034F9019B0133B3
:1035500005D18023044ADB0411680B43136000206B
:103560000EBDC0461C18001114F00040F0B5050057
:103570002026184B87B00493049B002B03D1112401
:10358000200007B0F0BD002102220B000191009144
:10359000052000F03DFC02230F490A681A42FCD1C5
:1035A0000596059C631E0593002CFAD10B4A1368FF
:1035B000002BFCDA0F276F440121380000F098FD42
:1035C0003B782B42DCD0052000F042FC049B013B01
:1035D0000493D1E7FFFFFF0790C8004000C80040F8
:1035E00007B500F0A5FC80220821D205936A01915D
:1035F000002B01D10739916202210C4A1160019917
:10360000481E01900029FAD1033111600531019162
:103610000199481E01900029FAD11160002B02D1B6
:103620008022D205936200F0EBFB07BD00C0004092
:10363000F0B52D4C89B02378002B4FD1FEF762F9FD
:1036400002232A4F03903A681A42FCD120230693A2
:10365000069B5A1E0692002BFAD1254E3368002B8A
:10366000FCDA0120FFF782FF011E02D0112009B011
:10367000F0BD030003220190009005AD9F2000F0F3
:10368000C7FB0321280000F033FD02233A681A42E9
:10369000FCD120230793079B5A1E0792002BFAD1D7
:1036A0003368002BFCDA0120FFF760FF0028DDD132
:1036B0000398FEF73BF9AA786B7811041B020B43C1
:1036C00029780B4363601300113B0A49052B07D887
:1036D00001239340A3600B60012323700020C6E701
:1036E00080231B03F6E7C0463445FF1F90C8004007
:1036F00000C800409808FF1F1E4B30B55A68187864
:103700001D4B85B0D31859424B4101210093002332
:1037100000F086FB194B1A4A02259A6300221A65AB
:1037200010325A658022C4219D65164B1648D2027C
:10373000DA6789004258154B80241A4080231B0405
:1037400013434350642341200393E40500F078F9C8
:10375000402000F075F96562039D6B1E0393002DF8
:10376000FAD103236362FFF73BFFA562FFF760FF17
:1037700005B030BD4045FF1F95FFFEF700C8004073
:10378000050001FF04E100E000E100E0FFFF00FFB1
:1037900010B5064B18705960FFF7AEFF00211320DB
:1037A000034AFFF7B1FD002010BDC0464045FF1F92
:1037B000F936FF1FF0B5040085B003920291FEF7C1
:1037C000A1F8882263035B0B52051A438023DB05B3
:1037D0009D6A8023274F0092BA68002601901B0340
:1037E0009A420CD9F82326001B041E401C4206D026
:1037F0008022214B52025E6219680A431A60002D32
:103800000BD100F095FB02221C4B1A608023DB05D4
:103810005A62013A9A6200F0F3FA0023039A934243
:1038200020D1002D0AD100F083FB144B03221D6030
:103830008023DB055A629D6200F0E2FA8023BA68B9
:103840001B039A4208D9002E06D000220A4B0C49CD
:103850005A621A680A401A600198FEF767F8002059
:1038600005B0F0BD009A0299D2181278CA540133FB
:10387000D4E7C0463445FF1F00C8004000C00040E8
:10388000FFFFFEFFF0B587B0029103920400FEF740
:1038900039F8019000F04CFB802302250122234ED1
:1038A000DB0535605D629A6200F0AAFA204F3B6842
:1038B0002B42FCD120230493049B5A1E0492002B1C
:1038C000FAD11C4D2B68002BFCDA0120FFF74EFECD
:1038D000002802D0112007B0F0BD2000039A029901
:1038E00000F02EFA022304003A681A42FCD1202389
:1038F0000593059B5A1E0592002BFAD12B68002BCD
:10390000FCDA0120FFF732FE051EE3D100F010FBC8
:1039100080230322DB0535605A629D6200F070FA55
:103920000198FEF703F8E0B2D5E7C04600C00040BA
:1039300090C8004000C80040F0B5802687B0040061
:10394000FDF7E0FFF605B36A02250393029000F04D
:10395000EFFA0123244F3D607562B36200F050FA24
:10396000224E33682B42FCD120230493049B5A1E21
:103970000492002BFAD11E4D2B68002BFCDA01209B
:10398000FFF7F4FD002802D0112007B0F0BD2000A1
:1039900000F0EEFB0223019032681A42FCD1202392
:1039A0000593059B5A1E0592002BFAD12B68002B1C
:1039B000FCDA0320FFF7DAFD041EE5D100F0B8FAC7
:1039C00080230322DB053C605A629C6200F018FAF7
:1039D000039B002B01D1FFF703FE0298FDF7A6FF22
:1039E0006B461879D1E7C04600C0004090C800403F
:1039F00000C8004007B5000201910422000A01A995
:103A0000FFF740FF0EBD000073B5050005240B4A0B
:103A1000A3005B429B1819686B46DE1D300000F066
:103A20005FFB022804D133782B55013CEFD276BDE1
:103A3000052CFCD00128FAD10230F8E71409001156
:103A40001F2807D8012380228340D20591680B43A9
:103A5000936070473F2808D8012380222038834094
:103A6000D20551690B435361F3E75F28F1D8012375
:103A7000802240388340D205116A0B431362E8E785
:103A80001F2807D8012280218240C9058B689343F3
:103A90008B6070473F2808D801228021203882405F
:103AA000C9054B6993434B61F3E75F28F1D80122C5
:103AB000802140388240C9050B6A93430B62E8E7D6
:103AC0001F2810D880230200DB05153A1968012A47
:103AD00006D820229143196019680A431A6070477A
:103AE00001228240F6E73F2811D880230200DB053F
:103AF000353AD968032A06D810229143D960D9688B
:103B00000A43DA60EBE7012220388240F5E75F28BC
:103B1000E5D842238022181A413B8340D205516ADE
:103B200099435162516A0B435362D8E710B50400C0
:103B3000012813D1A022184992050B685B015B098B
:103B400013430B60154B164A19681140154A0A4376
:103B50001A60402219680A431A6010BD0028FCD17F
:103B600001000A2000F07CFA21000B2000F078FA16
:103B7000C0220A4B920019680A4340211A601A6851
:103B80008A431A60B022044912060B685B015B0984
:103B900013430B60E1E7C04614F000401CF0004006
:103BA0007F00FEFF80FD010072B6074A13680133F3
:103BB00013600422054B1A600023054A136080221B
:103BC000D2055360FEE7C0467808FF1FC0F00040F2
:103BD000C4F00040044B054A1A60054B1A600022ED
:103BE000044B1A607047C046140AFF1F841E000071
:103BF000380AFF1FC4F000400023034A1360034A41
:103C00001360034A1360704754F0004040F10040D5
:103C100044F10040002310B5184C8AB00093019382
:103C20002378012B27D06946012000F0F1F9002804
:103C300017D1009B12490293019B06AA0393114BD3
:103C400002A81B680493104B1B68059300F0A8F9A9
:103C500010220E4906A800F0EBF8002804D1FF233B
:103C6000237000200AB010BD0123094A074902A8A9
:103C7000237000F095F90120F4E7C0465C66FF1F51
:103C800010290011082900110C2900112029001108
:103C90006066FF1F13B501246946012000F0B8F9E2
:103CA000034B00940193FFF7B5FF200016BDC046FB
:103CB000BB0B000010B5FFF79FFFFFF7EBFF0028DD
:103CC00002D0024B984710BDFEE7C046E1A20000BB
:103CD00002B4714649084900095649008E4402BCA5
:103CE0007047C04602B4714649084900095C490062
:103CF0008E4402BC7047C04603B471464908400078
:103D00004900095A49008E4403BC70470000000076
:103D100001B40248844601BC604700BFF53501008C
:103D200001B40248844601BC604700BFF9ED0000C1
:103D300001B40248844601BC604700BF61370100FE
:103D400001B40248844601BC604700BF957301007E
:103D500001B40248844601BC604700BF116E0000F8
:103D600001B40248844601BC604700BF89140100C9
:103D700001B40248844601BC604700BF894400008A
:103D800001B40248844601BC604700BFF9A60000A8
:103D900001B40248844601BC604700BF8D82000028
:103DA00001B40248844601BC604700BFD9B000009E
:103DB00001B40248844601BC604700BFC1F700005F
:103DC00001B40248844601BC604700BFE9270000F7
:103DD00001B40248844601BC604700BFB70E000032
:103DE00001B40248844601BC604700BF2D6C01004D
:103DF00001B40248844601BC604700BF21A900000D
:103E000001B40248844601BC604700BF9DA9000080
:103E100001B40248844601BC604700BF496D0100FF
:103E200001B40248844601BC604700BFC56D010073
:103E300001B40248844601BC604700BFCD4C01007C
:103E400001B40248844601BC604700BFF90D01007F
:103E500001B40248844601BC604700BF01890000EC
:103E600001B40248844601BC604700BFED6B01000D
:103E700001B40248844601BC604700BF7997000046
:103E800001B40248844601BC604700BF6DF60000E3
:103E900001B40248844601BC604700BF156B0100B5
:103EA00001B40248844601BC604700BFE9F6000047
:103EB00001B40248844601BC604700BF5976010046
:103EC00001B40248844601BC604700BFBD5C0100EC
:103ED00001B40248844601BC604700BFC11501001F
:103EE00001B40248844601BC604700BF05340100AC
:103EF00001B40248844601BC604700BF016701006D
:103F000001B40248844601BC604700BF7912010039
:103F100001B40248844601BC604700BF9D6A0000AE
:103F200001B40248844601BC604700BFE9170100A4
:103F300001B40248844601BC604700BF75A9000077
:103F400001B40248844601BC604700BF01D70000AD
:103F500001B40248844601BC604700BF9DB2001115
:103F600001B40248844601BC604700BF016C0100F7
:103F700001B40248844601BC604700BF75F80000E8
:103F800001B40248844601BC604700BFF935010016
:103F900001B40248844601BC604700BF090E00001E
:103FA00001B40248844601BC604700BFDD3F000009
:103FB00001B40248844601BC604700BF8D11010076
:103FC00001B40248844601BC604700BFE9D4000048
:103FD00001B40248844601BC604700BFBD0B01002C
:103FE00001B40248844601BC604700BFE94C0100AF
:103FF00001B40248844601BC604700BF51B80000CC
:1040000001B40248844601BC604700BF8937010003
:1040100001B40248844601BC604700BFE1AC000027
:1040200001B40248844601BC604700BFED6801004E
:1040300001B40248844601BC604700BF090E00007D
:1040400001B40248844601BC604700BFADAE000029
:1040500001B40248844601BC604700BFB35201006E
:1040600001B40248844601BC604700BF8D9E001128
:1040700001B40248844601BC604700BFE51201005C
:1040800001B40248844601BC604700BFE90B01004F
:1040900001B40248844601BC604700BFCD0C01005A
:1040A00001B40248844601BC604700BF8B52010046
:1040B00001B40248844601BC604700BF21440000AF
:1040C00001B40248844601BC604700BF19FA0000F1
:1040D00001B40248844601BC604700BF19070100D3
:1040E00001B40248844601BC604700BF8D3800110E
:1040F00001B40248844601BC604700BF3D71010025
:1041000001B40248844601BC604700BFDD0C0100D9
:1041100001B40248844601BC604700BF0D52010053
:1041200001B40248844601BC604700BF85C100005D
:1041300001B40248844601BC604700BF013401005D
:1041400001B40248844601BC604700BF85120100EB
:1041500001B40248844601BC604700BFDD0A01008B
:1041600001B40248844601BC604700BF0934010025
:1041700001B40248844601BC604700BFA96F01003A
:1041800001B40248844601BC604700BFC1A50000DD
:1041900001B40248844601BC604700BFA9D80000B2
:1041A00001B40248844601BC604700BFEDA5000091
:1041B00001B40248844601BC604700BFD5440100F9
:1041C00001B40248844601BC604700BF4DF90000BD
:1041D00001B40248844601BC604700BF855201001B
:1041E00001B40248844601BC604700BF53B90000D7
:1041F00001B40248844601BC604700BF6D0B01005A
:1042000001B40248844601BC604700BFC16601009A
:1042100001B40248844601BC604700BF71B0000091
:1042200001B40248844601BC604700BFC95C01007C
:1042300001B40248844601BC604700BF6911010017
:1042400001B40248844601BC604700BFC9A9000010
:1042500001B40248844601BC604700BFA1AF000022
:1042600002000000D2BB001101000000A0B9001143
:1042700002000000CEBB001101000000A042FF1FA1
:1042800002000000A8B9001101000000A463FF1F94
:1042900002000000CCBB0011030000001863FF1FE8
:1042A0001200000002000000D2BB0011010000005B
:1042B000E8B9001102000000CEBB001101000000AF
:1042C000E5B9001102000000F2B90011030000007E
:1042D0005363FF1F02000000CCBB0011030000006D
:1042E0006863FF1F02000000CEBB00110100000048
:1042F000E4B9001102000000F0B900110300000051
:104300002963FF1F02000000CCBB00110300000066
:104310004A63FF1F02000000D2BB00110100000031
:104320002CBA001102000000CEBB001101000000F9
:10433000E943FF1F020000003EBA00110100000027
:1043400023BA001102000000CEBB001101000000E2
:10435000E843FF1F020000003CBA0011010000000A
:104360007063FF1F02000000CEBB001101000000BF
:10437000E743FF1F020000003ABA001101000000ED
:1043800013BA001102000000CEBB001101000000B2
:10439000E643FF1F0200000038BA001101000000D0
:1043A0000EBA001102000000CEBB00110100000097
:1043B000E543FF1F0200000036BA001101000000B3
:1043C00009BA001102000000CEBB0011010000007C
:1043D000E443FF1F0200000034BA00110100000096
:1043E00004BA001102020202020200008D4B001109
:1043F000514B001180BA0011900118001800FFFF06
:104400000701020304050602010600000000000087
:10441000000000000000000000000000000000009C
:10442000000000000000030002000000D2BB0011E9
:104430000100000000BB001102000000CEBB001113
:10444000010000009844FF1F020000000ABB001199
:10445000010000009E63FF1F02000000CCBB0011A2
:10446000030000000C66FF1F02000000CEBB00111D
:10447000010000009844FF1F0200000008BB00116B
:1044800001000000A063FF1F02000000CCBB001170
:10449000030000000466FF1F12000000000100007E
:1044A00000000111FFFF00005048593600000000D5
:1044B000000000000100000091BA00110B0005008F
:1044C000F7000000B4000028002800283075A00084
:1044D000A000A000A00000080008E001F00010000B
:1044E000100010001000100010005000500050008C
:1044F00010001000D0070000000000000F000100B5
:104500000500307507001000010081FF0000000069
:10451000FF000000657000116D6E0011FD6B001151
:10452000FFFF0100FF000000819A0011FD970011BC
:1045300015970011000000000000000000000800B6
:10454000040000003B0001085902E0018821280016
:10455000FF00000002000000D2BB001101000000BB
:1045600098BC001102000000CEBB00110100000049
:10457000D145FF1F02000000CABB0011010000006E
:10458000186AFF1F02000000CEBB001101000000EE
:10459000D045FF1F02000000C8BB00110100000051
:1045A000CE45FF1F02000000CEBB0011010000003D
:1045B000CC45FF1F02000000C6BB00110100000037
:1045C000C445FF1F180018000000900102000003FE
:1045D0000202000002000000D2BB00110100000036
:1045E000ACBC001102000000CEBB001101000000B5
:1045F0001446FF1F02000000C4BB001100000000B1
:104600000000000002000000CCBB0011030000000D
:06461000386AFF1F20FFC5
:040000051FFF184180
:00000001FF
